:020000040000FA
:0408000055EF0BF0B5
:1008100003B272EF05F0F2B490EF05F09EB098EFDE
:1008200005F09EB2A0EF05F0F2A81AEF04F0F2B2C4
:1008300021EF04F0F2B01FEF04F004EF0BF0F2969A
:10084000F290CD90F2929EA02BEF04F00101533F65
:100850002BEF04F0542BAEC1B2F1AFC1B3F1B0C174
:10086000B4F1B1C1B5F1AAC1AEF1ABC1AFF1ACC148
:10087000B0F1ADC1B1F1A6C1AAF1A7C1ABF1A8C158
:10088000ACF1A9C1ADF1A2C1A6F1A3C1A7F1A4C168
:10089000A8F1A5C1A9F19EC1A2F19FC1A3F1A0C178
:1008A000A4F1A1C1A5F19AC19EF19BC19FF19CC188
:1008B000A0F19DC1A1F196C19AF197C19BF198C198
:1008C0009CF199C19DF1CECF96F1CFCF97F153C155
:1008D00098F154C199F1CF6ACE6A0101536B546B00
:1008E0009E90CD800FBC0F8E0FBA7AEF04F00F8A66
:1008F00004EF0BF00F8C0FBEB6EF04F096C19AF127
:1009000097C19BF198C19CF199C19DF19AC19EF14B
:100910009BC19FF19CC1A0F19DC1A1F19EC1A2F11B
:100920009FC1A3F1A0C1A4F1A1C1A5F1A2C1A6F1EB
:10093000A3C1A7F1A4C1A8F1A5C1A9F1A6C1AAF1BB
:10094000A7C1ABF1A8C1ACF1A9C1ADF1AAC1AEF18B
:10095000ABC1AFF1ACC1B0F1ADC1B1F1AEC1B2F15B
:10096000AFC1B3F1B0C1B4F1B1C1B5F101015E6B7A
:100970005F6B606B616B96515E2797515F23985157
:100980006023995161239A515E279B515F239C51AB
:1009900060239D5161239E515E279F515F23A0518B
:1009A0006023A1516123A2515E27A3515F23A4516B
:1009B0006023A5516123A6515E27A7515F23A8514B
:1009C0006023A9516123AA515E27AB515F23AC512B
:1009D0006023AD516123AE515E27AF515F23B0510B
:1009E0006023B1516123B2515E27B3515F23B451EB
:1009F0006023B5516123D8900101613360335F33C7
:100A00005E33D8900101613360335F335E33D89039
:100A10000101613360335F335E3300C10CF101C10A
:100A20000DF102C10EF103C10FF104C110F105C1B6
:100A300011F106C112F107C113F108C114F109C186
:100A400015F10AC116F10BC117F134C135F111B816
:100A500035EF05F00101620E046F010E056F000E07
:100A6000066F000E076F3EEF05F00101A70E046F41
:100A7000020E056F000E066F000E076F5EC100F1DB
:100A80005FC101F160C102F161C103F13DEC2CF0E5
:100A900003BF04D019BE02D019A0108C11A056EFCC
:100AA00005F010BA56EF05F00F80108A0CC100F166
:100AB0000DC101F10EC102F10FC103F110C104F12A
:100AC00011C105F112C106F113C107F114C108F1FA
:100AD00015C109F116C10AF117C10BF135C134F185
:100AE00004EF0BF00392ABB2AB98AB88030103EEBB
:100AF00000F080517F0BE92604C0EFFF802B81516D
:100B0000805D700BD8A48B8200008051815D700BDA
:100B1000D8A48B9281518019D8B4079004EF0BF0C0
:100B2000F2940101453F04EF0BF0462B04EF0BF06C
:100B30009E900101533F04EF0BF0542B04EF0BF098
:100B40009E9211B823EF08F0040066A1A8EF05F00B
:100B50008BB4B2EF05F010ACB2EF05F08B84109CB3
:100B6000B3EF05F08B94077C07ACCEEF05F0C274B1
:100B7000C2B4C8EF05F0C3CFB7F5C4CFB8F50501CF
:100B8000D890B833B733D890B833B733CFEF05F038
:100B9000C3CF55F1C4CF56F1CFEF05F0C28207B4F1
:100BA0003CEF06F047C14BF148C14CF149C14DF152
:100BB0004AC14EF15EC162F15FC163F160C164F18F
:100BC00061C165F196C1B6F197C1B7F198C1B8F1AD
:100BD00099C1B9F19AC1BAF19BC1BBF19CC1BCF1F9
:100BE0009DC1BDF19EC1BEF19FC1BFF1A0C1C0F1C9
:100BF000A1C1C1F1A2C1C2F1A3C1C3F1A4C1C4F199
:100C0000A5C1C5F1A6C1C6F1A7C1C7F1A8C1C8F168
:100C1000A9C1C9F1AAC1CAF1ABC1CBF1ACC1CCF138
:100C2000ADC1CDF1AEC1CEF1AFC1CFF1B0C1D0F108
:100C3000B1C1D1F1B2C1D2F1B3C1D3F1B4C1D4F1D8
:100C4000B5C1D5F1B7C5B9F5B8C5BAF5B9C5BBF5E4
:100C5000BAC5BCF5010155515B2756515C23E86AC2
:100C60005D230E2E3CEF06F05CC157F15DC158F1DB
:100C70005B6B5C6B5D6B078E0201002F04EF0BF06A
:100C80003C0E006F1A50E00BE00AE866128818BEAE
:100C900002D018B4108E00C10CF101C10DF102C1D7
:100CA0000EF103C10FF104C110F105C111F106C12C
:100CB00012F107C113F108C114F109C115F10AC1FC
:100CC00016F10BC117F134C135F181AA1CEF07F001
:100CD00030A0EDEF06F005012F51000AD8B41CEF4B
:100CE00007F005012F51010AD8B4A6EF06F005015F
:100CF0002F51020AD8B4E7EF06F005012F51030A7D
:100D0000D8B4E7EF06F005012F51040AD8B4E7EF95
:100D100006F005012F51050AD8B4E7EF06F00501EA
:100D20002F51060AD8B4E7EF06F005012F51070A44
:100D3000D8B4E7EF06F005012F51320AD8B4A4EF7A
:100D400006F02F6B1CEF07F01CEF07F0050157674B
:100D5000B1EF06F05867B1EF06F05967B1EF06F052
:100D60005A67B5EF06F01CEF07F05BC500F15CC5F4
:100D700001F15DC502F15EC503F10101010E046FD1
:100D8000000E056F000E066F000E076F3DEC2CF095
:100D900000C15BF501C15CF502C15DF503C15EF503
:100DA0000067DAEF06F00167DAEF06F00267DAEFC4
:100DB00006F003671CEF07F057C55BF558C55CF5F7
:100DC00059C55DF55AC55EF50F881CEF07F00501A2
:100DD0003067EDEF06F01CEF07F00FBE02EF07F0F3
:100DE00010A007EF07F001014767FEEF06F0486724
:100DF000FEEF06F04967FEEF06F04A6702EF07F0E4
:100E000007EF07F007AE07EF07F019EF07F005014E
:100E1000312F1CEF07F03C0E316F302F1CEF07F025
:100E20000101000E626FE00E636FA50E646F010E8C
:100E3000656F0501306B0F880501666B37B722EFD0
:100E400007F066810CC100F10DC101F10EC102F184
:100E50000FC103F110C104F111C105F112C106F176
:100E600013C107F114C108F115C109F116C10AF146
:100E700017C10BF135C134F100C10CF101C10DF105
:100E800002C10EF103C10FF104C110F105C111F14E
:100E900006C112F107C113F108C114F109C115F11E
:100EA0000AC116F10BC117F134C135F101018A678E
:100EB00061EF07F08B6761EF07F08C6761EF07F078
:100EC0008D6765EF07F095EF07F08EC100F18FC1D8
:100ED00001F190C102F191C103F10101010E046F12
:100EE000000E056F000E066F000E076F3DEC2CF034
:100EF00000C18EF101C18FF102C190F103C191F1E6
:100F000000678AEF07F001678AEF07F002678AEF50
:100F100007F0036795EF07F08AC18EF18BC18FF15F
:100F20008CC190F18DC191F10F80D57ED5BE6DD071
:100F3000D6CF47F1D7CF48F145C149F1E86AE8CFAC
:100F40004AF119BE02D019A0108C109047C100F1CF
:100F500048C101F149C102F14AC103F101010A0E80
:100F6000046F000E056F000E066F000E076F3DEC5C
:100F70002CF003AF1080010154A7CBEF07F00F9ABC
:100F80000F9C0F9E0101000E5E6F600E5F6F3D0EA5
:100F9000606F080E616F010147BFDBEF07F0486724
:100FA000DBEF07F04967DBEF07F04A67DBEF07F09D
:100FB000F28800EF08F0F2985E6B5F6B606B616B1C
:100FC000966B976B986B996B9A6B9B6B9C6B9D6BFD
:100FD0009E6B9F6BA06BA16BA26BA36BA46BA56BAD
:100FE000A66BA76BA86BA96BAA6BAB6BAC6BAD6B5D
:100FF000AE6BAF6BB06BB16BB26BB36BB46BB56B0D
:10100000D76AD66A0101456B466B0CC100F10DC170
:1010100001F10EC102F10FC103F110C104F111C1C0
:1010200005F112C106F113C107F114C108F115C190
:1010300009F116C10AF117C10BF135C134F104EF02
:101040000BF004EF0BF00201002F6DEF0AF0D59EBC
:10105000D6CF47F1D7CF48F145C149F1E86AE8CF8B
:101060004AF1D76AD66A0101456B466BD58E1A5094
:10107000E00BE00AE866128818BE02D018B4108EA1
:1010800017AE1C8C00C10CF101C10DF102C10EF1B3
:1010900003C10FF104C110F105C111F106C112F134
:1010A00007C113F108C114F109C115F10AC116F104
:1010B0000BC117F134C135F10FA0109A11B86CEFC4
:1010C00008F00101620E046F010E056F000E066F3D
:1010D000000E076F75EF08F00101A70E046F020EF6
:1010E000056F000E066F000E076F47C100F148C183
:1010F00001F149C102F14AC103F13DEC2CF003BFFB
:1011000088EF08F019BE02D019A0108C11B00F8022
:101110000CC100F10DC101F10EC102F10FC103F1CB
:1011200010C104F111C105F112C106F113C107F19B
:1011300014C108F115C109F116C10AF117C10BF16B
:1011400035C134F102013C0E006F00C10CF101C148
:101150000DF102C10EF103C10FF104C110F105C17F
:1011600011F106C112F107C113F108C114F109C14F
:1011700015F10AC116F10BC117F134C135F181AA7D
:1011800076EF09F030A047EF09F005012F51000A72
:10119000D8B476EF09F005012F51010AD8B400EF59
:1011A00009F005012F51020AD8B441EF09F00501F9
:1011B0002F51030AD8B441EF09F005012F51040A59
:1011C000D8B441EF09F005012F51050AD8B441EF19
:1011D00009F005012F51060AD8B441EF09F00501C5
:1011E0002F51070AD8B441EF09F005012F51320AF7
:1011F000D8B4FEEF08F02F6B76EF09F076EF09F028
:10120000050157670BEF09F058670BEF09F05967B5
:101210000BEF09F05A670FEF09F076EF09F05BC5A5
:1012200000F15CC501F15DC502F15EC503F101018C
:10123000010E046F000E056F000E066F000E076FA3
:101240003DEC2CF000C15BF501C15CF502C15DF520
:1012500003C15EF5006734EF09F0016734EF09F070
:10126000026734EF09F0036776EF09F057C55BF5C5
:1012700058C55CF559C55DF55AC55EF50F8876EF22
:1012800009F00501306747EF09F076EF09F00FBE6E
:101290005CEF09F010A061EF09F00101476758EF1A
:1012A00009F0486758EF09F0496758EF09F04A67B5
:1012B0005CEF09F061EF09F007AE61EF09F073EF41
:1012C00009F00501312F76EF09F03C0E316F302F18
:1012D00076EF09F00101000E626FE00E636FA50E5C
:1012E000646F010E656F0501306B0F880501666B39
:1012F00037B77CEF09F066810CC100F10DC101F137
:101300000EC102F10FC103F110C104F111C105F1C9
:1013100012C106F113C107F114C108F115C109F199
:1013200016C10AF117C10BF135C134F100C10CF13E
:1013300001C10DF102C10EF103C10FF104C110F1A1
:1013400005C111F106C112F107C113F108C114F171
:1013500009C115F10AC116F10BC117F134C135F1FC
:1013600001018A67BBEF09F08B67BBEF09F08C675F
:10137000BBEF09F08D67BFEF09F0EFEF09F08EC109
:1013800000F18FC101F190C102F191C103F101019E
:10139000010E046F000E056F000E066F000E076F42
:1013A0003DEC2CF000C18EF101C18FF102C190F132
:1013B00003C191F10067E4EF09F00167E4EF09F080
:1013C0000267E4EF09F00367EFEF09F08AC18EF1DD
:1013D0008BC18FF18CC190F18DC191F10F80109074
:1013E00047C100F148C101F149C102F14AC103F10D
:1013F00001010A0E046F000E056F000E066F000E4D
:10140000076F3DEC2CF003AF1080010154A715EFDE
:101410000AF00F9A0F9C0F9E0101000E5E6F600E86
:101420005F6F3D0E606F080E616F47C100F148C1EC
:1014300001F149C102F14AC103F10101140E046F27
:10144000050E056F000E066F000E076F3DEC2CF0C9
:1014500003AF2EEF0AF0F28853EF0AF0F2985E6BBA
:101460005F6B606B616B966B976B986B996B9A6B0C
:101470009B6B9C6B9D6B9E6B9F6BA06BA16BA26B20
:10148000A36BA46BA56BA66BA76BA86BA96BAA6BD0
:10149000AB6BAC6BAD6BAE6BAF6BB06BB16BB26B80
:1014A000B36BB46BB56B0CC100F10DC101F10EC192
:1014B00002F10FC103F110C104F111C105F112C114
:1014C00006F113C107F114C108F115C109F116C1E4
:1014D0000AF117C10BF135C134F104008BB478EF78
:1014E0000AF010AC78EF0AF08B84109C79EF0AF0C8
:1014F0008B94077C07AC94EF0AF0C274C2B48EEFF1
:101500000AF0C3CFB7F5C4CFB8F50501D890B8330A
:10151000B733D890B833B73395EF0AF0C3CF55F14E
:10152000C4CF56F195EF0AF0C28207B402EF0BF078
:1015300047C14BF148C14CF149C14DF14AC14EF18F
:101540005EC162F15FC163F160C164F161C165F1C7
:1015500096C1B6F197C1B7F198C1B8F199C1B9F187
:101560009AC1BAF19BC1BBF19CC1BCF19DC1BDF157
:101570009EC1BEF19FC1BFF1A0C1C0F1A1C1C1F127
:10158000A2C1C2F1A3C1C3F1A4C1C4F1A5C1C5F1F7
:10159000A6C1C6F1A7C1C7F1A8C1C8F1A9C1C9F1C7
:1015A000AAC1CAF1ABC1CBF1ACC1CCF1ADC1CDF197
:1015B000AEC1CEF1AFC1CFF1B0C1D0F1B1C1D1F167
:1015C000B2C1D2F1B3C1D3F1B4C1D4F1B5C1D5F137
:1015D000B7C5B9F5B8C5BAF5B9C5BBF5BAC5BCF557
:1015E000010155515B2756515C23E86A5D230E2E9D
:1015F00002EF0BF05CC157F15DC158F15B6B5C6BA6
:101600005D6B078E04EF0BF002C0E0FF005001C0DD
:10161000D8FF1000A6B20AEF0BF00CC0A9FF0BC058
:10162000A8FFA69EA69CA684F29E550EA76EAA0EA3
:10163000A76EA682F28EA694A6B21CEF0BF00C2A1F
:101640001200A96EA69EA69CA680A8500C2A120085
:1016500004012C0E826F73EC0EF038EC2DF00C5060
:1016600021EC0BF0E8CF00F10C5021EC0BF0E8CFAF
:1016700001F101AF41EF0BF00101FF0E026FFF0E10
:10168000036FDBEC2CF029674DEF0BF00401200E0B
:10169000826F73EC0EF052EF0BF004012D0E826F8F
:1016A00073EC0EF0E5EC2AF01200306A076A0F6A5C
:1016B000106A116A126A136A0F010D0EC16E860E4E
:1016C000C06E030EC26E0F01680E896E130E926E0D
:1016D000080E8A6EF30E936E8B6A900E946EC80E8F
:1016E00021EC0BF0E8CFE8FF1098E8A0108810A8D4
:1016F00005D00E0E226E8E0E236E04D00F0E226EBB
:101700008F0E236EB7EC2DF0F18EF19EFC0E21ECC6
:101710000BF0E8CF0BF00BA011800BA211820BA4F1
:1017200011840BA81188C90E21EC0BF0E8CF17F03B
:10173000CA0E21EC0BF0E8CF18F0CB0E21EC0BF029
:10174000E8CF19F0CC0E21EC0BF0E8CF1AF0CD0E5B
:1017500021EC0BF0E8CF2FF01C6A1D6A0E6A010124
:101760005B6B5C6B5D6B576B586BF29A0101476B5F
:10177000486B496B4A6B4B6B4C6B4D6B4E6B4F6BB5
:10178000506B516B526B456B466BD76AD66A0F0133
:10179000280ED56EF28A9D90B00ECD6E01015E6B63
:1017A0005F6B606B616B626B636B646B656B666BCD
:1017B000676B686B696B536B546BCF6ACE6A0F9A19
:1017C0000F9C0F9E9D80760ECA6E9D8202013C0E7C
:1017D000006FCC6A160E21EC0BF0E8CF00F1170E6B
:1017E00021EC0BF0E8CF01F1180E21EC0BF0E8CF63
:1017F00002F1190E21EC0BF0E8CF03F1010103AF68
:101800001CEF0CF038EC2DF0160E0C6E00C10BF036
:101810000AEC0BF0170E0C6E01C10BF00AEC0BF08A
:10182000180E0C6E02C10BF00AEC0BF0190E0C6EC8
:1018300003C10BF00AEC0BF000C18AF101C18BF17E
:1018400002C18CF103C18DF100C18EF101C18FF194
:1018500002C190F103C191F11A0E21EC0BF0E8CF17
:1018600000F11B0E21EC0BF0E8CF01F11C0E21EC76
:101870000BF0E8CF02F11D0E21EC0BF0E8CF03F1E5
:10188000010103AF72EF0CF038EC2DF01A0E0C6E64
:1018900000C10BF00AEC0BF01B0E0C6E01C10BF03B
:1018A0000AEC0BF01C0E0C6E02C10BF00AEC0BF0F4
:1018B0001D0E0C6E03C10BF00AEC0BF01A0E21EC9E
:1018C0000BF0E8CF00F11B0E21EC0BF0E8CF01F19B
:1018D0001C0E21EC0BF0E8CF02F11D0E21EC0BF0F9
:1018E000E8CF03F100C192F101C193F102C194F17B
:1018F00003C195F1240EAC6E900EAB6E240EAC6E4F
:10190000080EB86E000EB06E1F0EAF6E0401806B35
:10191000816B0F01900EAB6E0F019D8A0301806BEE
:10192000816BC26B8B925BEC32F05BEC32F0B9EC0A
:1019300033F03AEC30F0200E21EC0BF0E8CF2FF52D
:1019400005012F51FF0AD8A4ADEF0CF02F6B200E2C
:101950000C6E2FC50BF00AEC0BF00501010E306F79
:101960003C0E316F250E21EC0BF0E8CF00F1260E76
:1019700021EC0BF0E8CF01F1270E21EC0BF0E8CFC2
:1019800002F1280E21EC0BF0E8CF03F1010103AFC7
:10199000E4EF0CF038EC2DF0250E0C6E00C10BF0CE
:1019A0000AEC0BF0260E0C6E01C10BF00AEC0BF0EA
:1019B000270E0C6E02C10BF00AEC0BF0280E0C6E19
:1019C00003C10BF00AEC0BF000C157F501C158F54B
:1019D00002C159F503C15AF500C15BF501C15CF5BF
:1019E00002C15DF503C15EF5290E21EC0BF0E8CFD5
:1019F0005FF5050160515F5DD8A05FC560F5210E00
:101A000021EC0BF0E8CF00F1220E21EC0BF0E8CF37
:101A100001F1230E21EC0BF0E8CF02F1240E21ECB2
:101A20000BF0E8CF03F1010103AF45EF0DF038EC07
:101A30002DF0210E0C6E00C10BF00AEC0BF0220E03
:101A40000C6E01C10BF00AEC0BF0230E0C6E02C100
:101A50000BF00AEC0BF0240E0C6E03C10BF00AEC39
:101A60000BF0210E21EC0BF0E8CF00F1220E21EC5F
:101A70000BF0E8CF01F1230E21EC0BF0E8CF02F1DF
:101A8000240E21EC0BF0E8CF03F100C161F501C198
:101A900062F502C163F503C164F582EC2FF068ECD6
:101AA0002EF0C0EC2DF030A0B6EF0DF005012F5157
:101AB000020A16E005012F51030A19E005012F5112
:101AC000040A24E005012F51050A2BE005012F51DE
:101AD000060A39E005012F51070A3FE0B6EF0DF085
:101AE000602FB3EF0DF05FC560F5B6EF0DF0B0C538
:101AF00000F101010F0E001701010051000A36E04C
:101B000001010051050A32E0B3EF0DF0B0C500F15C
:101B100001010F0E001701010051000A27E0B3EF89
:101B20000DF00501B051000A21E00501B051150A80
:101B30001DE00501B051300A19E00501B051450A18
:101B400015E0B3EF0DF00501B051000A0FE00501FB
:101B5000B051300A0BE0B3EF0DF00501B051000AAF
:101B600005E0B3EF0DF081BAF8EF33F00790000114
:101B7000F28EF28C12AE03D012BCB2EF18F007B0A6
:101B80006BEF29F00FB0FFEF22F010BEFFEF22F055
:101B900012B8FFEF22F00FB89AEF1CF0030180514A
:101BA00081197F0BD8B46BEF29F013EE00F081514F
:101BB0007F0BE126812BE7CFE8FFE00BD8B46BEF7A
:101BC00029F023EE82F0C2513F0BD926E7CFDFFF89
:101BD000C22BDF50780AD8A46BEF29F007808EC1A2
:101BE00000F18FC101F190C102F191C103F1010136
:101BF000040E046F000E056F000E066F000E076FD7
:101C00003DEC2CF000AF0EEF0EF00101030E8E6FD5
:101C1000000E8F6F000E906F000E916F03018251C6
:101C2000720AD8B4E3EF22F08251520AD8B4E3EF3B
:101C300022F08251750AD8B4E3EF22F08251630A90
:101C4000D8B425EF26F08251690AD8B492EF1FF07C
:101C500082517A0AD8B4A5EF20F08251490AD8B44B
:101C600031EF1FF08251500AD8B44FEF1EF082516D
:101C7000700AD8B492EF1EF08251540AD8B4BDEF66
:101C80001EF08251740AD8B403EF1FF08251410A4A
:101C9000D8B489EF0FF082514B0AD8B487EF0EF019
:101CA00082516D0AD8B4BCEF13F082514D0AD8B4FA
:101CB000D5EF13F08251730AD8B413EF22F082519A
:101CC000530AD8B478EF22F082514C0AD8B464EFAA
:101CD00014F08251590AD8B40DEF13F012AE01D0AE
:101CE000128C5CEF26F0040114EE00F080517F0BA3
:101CF000E12682C4E7FF802B120004010D0E826FE3
:101D000073EC0EF00A0E826F73EC0EF012000401F9
:101D10004B0E826F73EC0EF004012C0E826F73EC8D
:101D20000EF081B802D02FB630D003018351430AA0
:101D3000D8B4CCEF0EF003018351630AD8B4CEEFD0
:101D40000EF003018351520AD8B4D0EF0EF0030114
:101D50008351720AD8B4D2EF0EF003018351470ABF
:101D6000D8B4D4EF0EF003018351670AD8B4D6EF8C
:101D70000EF003018351540AD8B4D8EF0EF00301DA
:101D80008351740AD8B447EF0FF003018351550A09
:101D9000D8B4DAEF0EF082D02F807AD02F9078D09E
:101DA0002F8276D02F9274D02F8472D02F9470D03F
:101DB0002F866ED084C330F185C331F186C332F1F2
:101DC00087C333F10101296B86EC2DF0FDEC2CF07B
:101DD00000C104F101C105F102C106F103C107F11F
:101DE00079EC2DF0200EF86EF76AF66A0900F5CF4F
:101DF0002CF10900F5CF2DF10900F5CF2EF10900E6
:101E0000F5CF2FF10900F5CF30F10900F5CF31F111
:101E10000900F5CF32F10900F5CF33F10101296B4B
:101E200086EC2DF0FDEC2CF03DEC2CF0006720EF63
:101E30000FF0016720EF0FF0026720EF0FF003674C
:101E400001D025D004014E0E826F73EC0EF0040118
:101E50006F0E826F73EC0EF004014D0E826F73EC07
:101E60000EF00401610E826F73EC0EF00401740E2B
:101E7000826F73EC0EF00401630E826F73EC0EF050
:101E80000401680E826F73EC0EF05AEF26F02F9665
:101E9000CD0E0C6E2FC00BF00AEC0BF0CD0E21EC2A
:101EA0000BF0E8CF2FF02FB006D00401630E826F45
:101EB00073EC0EF005D00401430E826F73EC0EF04C
:101EC0002FB206D00401720E826F73EC0EF005D0B3
:101ED0000401520E826F73EC0EF02FB406D0040191
:101EE000670E826F73EC0EF005D00401470E826F0F
:101EF00073EC0EF02FB606D00401740E826F73ECF3
:101F00000EF005D00401540E826F73EC0EF05AEF00
:101F100026F00401410E826F73EC0EF00301835131
:101F2000310AD8B42DEF12F003018351320AD8B42C
:101F30005DEF11F003018351330AD8B4E6EF10F0DE
:101F400003018351340AD8B4D6EF0FF00301835153
:101F5000350AD8B4B3EF0FF004013F0E826F73EC73
:101F60000EF05AEF26F004012C0E826F73EC0EF087
:101F700003018451300AD8B4C6EF0FF00301845135
:101F8000310AD8B4CEEF0FF01FEF11F08B9004019F
:101F9000300E826F73EC0EF0D4EF0FF08B800401E3
:101FA000310E826F73EC0EF05AEF26F0CC0E21EC5E
:101FB0000BF0E8CF0BF004012C0E826F73EC0EF0E7
:101FC00003018451310AD8B4FAEF0FF003018451B0
:101FD000300AD8B4FCEF0FF0030184514D0AD8B495
:101FE00006EF10F003018451540AD8B40DEF10F03D
:101FF00024EF10F08A8401D08A940BAE04D00BAC8D
:1020000002D00BBA21D0E00E0B1218D01F0E0B1607
:102010008539E844E00B0B1211D0E00E0B1679EC79
:102020002DF085C332F186C333F10101296B86ECB3
:102030002DF0FDEC2CF000511F0B0B12CC0E0C6E92
:102040000BC00BF00AEC0BF00401340E826F73EC42
:102050000EF004012C0E826F73EC0EF0CC0E21EC0E
:102060000BF0E8CF1AF08AB406D00401300E826F6C
:1020700073EC0EF005D00401310E826F73EC0EF09C
:1020800004012C0E826F73EC0EF01A38E840070B37
:10209000E8CF82F40401300E822773EC0EF00401C5
:1020A0002C0E826F73EC0EF038EC2DF01A501F0BD3
:1020B000E8CF00F1DBEC2CF032C182F40401300EE9
:1020C000822773EC0EF033C182F40401300E8227B4
:1020D00073EC0EF004012C0E826F73EC0EF038ECF2
:1020E0002DF02DC000F100AF0BD0FF0E016FFF0EE1
:1020F000026FFF0E036F04012D0E826F73EC0EF062
:10210000DBEC2CF031C182F40401300E822773EC39
:102110000EF032C182F40401300E822773EC0EF00F
:1021200033C182F40401300E822773EC0EF00401F7
:102130002C0E826F73EC0EF038EC2DF02CC000F1F9
:10214000DBEC2CF031C182F40401300E822773ECF9
:102150000EF032C182F40401300E822773EC0EF0CF
:1021600033C182F40401300E822773EC0EF00401B7
:102170002C0E826F73EC0EF038EC2DF02EC000F1B7
:1021800000AF0BD0FF0E016FFF0E026FFF0E036F4B
:1021900004012D0E826F73EC0EF0DBEC2CF031C1DC
:1021A00082F40401300E822773EC0EF032C182F407
:1021B0000401300E822773EC0EF033C182F4040167
:1021C000300E822773EC0EF05AEF26F0CB0E21EC86
:1021D0000BF0E8CF0BF004012C0E826F73EC0EF0C5
:1021E00003018451450AD8B40AEF11F00301845168
:1021F000440AD8B40DEF11F003018451300AD8B469
:1022000010EF11F003018451310AD8B414EF11F02A
:102210001FEF11F00B9E19EF11F00B8E19EF11F05B
:10222000FC0E0B1619EF11F0FC0E0B160B8019EFBC
:1022300011F0CB0E0C6E0BC00BF00AEC0BF004018E
:10224000330E826F73EC0EF004012C0E826F73EC70
:102250000EF0CB0E21EC0BF0E8CF19F019BE38EFE1
:1022600011F00401450E826F73EC0EF03DEF11F09A
:102270000401440E826F73EC0EF004012C0E826F89
:1022800073EC0EF00401300E826F73EC0EF004015B
:102290002C0E826F73EC0EF019B056EF11F00401A2
:1022A000300E826F73EC0EF05BEF11F00401310E13
:1022B000826F73EC0EF05AEF26F0CA0E21EC0BF091
:1022C000E8CF0BF004012C0E826F73EC0EF00301CB
:1022D0008451450AD8B499EF11F003018451440A9E
:1022E000D8B49CEF11F0030184514D0AD8B4A5EF86
:1022F00011F003018451410AD8B49FEF11F003019A
:102300008451460AD8B4A2EF11F003018451560A51
:10231000D8B4ADEF11F003018451500AD8B4B8EF2E
:1023200011F003018451520AD8B4BBEF11F0C4EF8D
:1023300011F00B9EBEEF11F00B8EBEEF11F00B9C57
:10234000BEEF11F00B8CBEEF11F0FC0E0B1685C327
:10235000E8FF030B0B12BEEF11F0C70E0B1685C37F
:10236000E8FF070BE846E846E8460B12BEEF11F01F
:102370000B84BEEF11F00B94BEEF11F0CA0E0C6E81
:102380000BC00BF00AEC0BF0CA0E21EC0BF0E8CFFF
:1023900018F00401320E826F73EC0EF004012C0E63
:1023A000826F73EC0EF018BEDDEF11F00401450EE4
:1023B000826F73EC0EF0E2EF11F00401440E826FB5
:1023C00073EC0EF004012C0E826F73EC0EF018C04B
:1023D000E8FF030BE8CF82F40401300E822773EC90
:1023E0000EF004012C0E826F73EC0EF018BC00EF9F
:1023F00012F00401410E826F73EC0EF005EF12F043
:102400000401460E826F73EC0EF004012C0E826FF5
:1024100073EC0EF018C0E8FF380BE842E842E842DF
:10242000E8CF82F40401300E822773EC0EF0040131
:102430002C0E826F73EC0EF018B426EF12F004012C
:10244000520E826F73EC0EF02BEF12F00401500E5F
:10245000826F73EC0EF05AEF26F0C90E21EC0BF0F0
:10246000E8CF0BF004012C0E826F73EC0EF0030129
:102470008451450AD8B44BEF12F003018451440A49
:10248000D8B44EEF12F0030184514D0AD8B451EF85
:1024900012F05FEF12F00B9E59EF12F00B8E59EF16
:1024A00012F0F80E0B1685C3E8FF070B0B1259EF5D
:1024B00012F0C90E0C6E0BC00BF00AEC0BF004010D
:1024C000310E826F73EC0EF004012C0E826F73ECF0
:1024D0000EF0C90E21EC0BF0E8CF17F017BE06D0B6
:1024E0000401450E826F73EC0EF005D00401440E1A
:1024F000826F73EC0EF004012C0E826F73EC0EF001
:1025000017C0E8FF070BE8CF82F40401300E8227E2
:1025100073EC0EF004012C0E826F73EC0EF007804A
:1025200038EC2DF028C0E8FF003B00430043030BCC
:10253000DBEC2CF033C182F40401300E822773EC03
:102540000EF004012C0E826F73EC0EF038EC2DF0BF
:1025500028C001F1019F019D29C000F10101DBECC0
:102560002CF02FC182F40401300E822773EC0EF0A0
:1025700030C182F40401300E822773EC0EF031C1B9
:1025800082F40401300E822773EC0EF032C182F423
:102590000401300E822773EC0EF033C182F4040183
:1025A000300E822773EC0EF004012C0E826F73EC58
:1025B0000EF038EC2DF02AC001F12BC000F1D890BC
:1025C00001330033D890013300330101DBEC2CF0F0
:1025D0002FC182F40401300E822773EC0EF030C15B
:1025E00082F40401300E822773EC0EF031C182F4C4
:1025F0000401300E822773EC0EF032C182F4040124
:10260000300E822773EC0EF033C182F40401300ED9
:10261000822773EC0EF05AEF26F0FC0E21EC0BF043
:10262000E8CF0BF003018351520AD8B444EF13F002
:1026300003018351720AD8B447EF13F003018351A9
:10264000500AD8B44AEF13F003018351700AD8B48A
:102650004DEF13F003018351550AD8B450EF13F036
:1026600003018351750AD8B453EF13F0030183516A
:10267000430AD8B45CEF13F003018351630AD8B462
:102680005FEF13F068EF13F00B9062EF13F00B8025
:1026900062EF13F00B9262EF13F00B8262EF13F014
:1026A0000B9462EF13F00B8462EF13F00B9662EF62
:1026B00013F00B8662EF13F00B9862EF13F00B88A8
:1026C00062EF13F0FC0E0C6E0BC00BF00AEC0BF07B
:1026D0000401590E826F73EC0EF011901192119457
:1026E0001198FC0E21EC0BF0E8CF0BF00BA0118041
:1026F0000BA211820BA411840BA8118811A088EFE2
:1027000013F00401520E826F73EC0EF08DEF13F094
:102710000401720E826F73EC0EF011A897EF13F0A4
:102720000401430E826F73EC0EF09CEF13F0040172
:10273000630E826F73EC0EF011A2A6EF13F004018A
:10274000500E826F73EC0EF0ABEF13F00401700EBD
:10275000826F73EC0EF011A4B5EF13F00401550E67
:10276000826F73EC0EF0BAEF13F00401750E826FF6
:1027700073EC0EF05AEF26F004016D0E826F73ECCD
:102780000EF003018351300AD8B414EF14F00301A2
:102790008351310AD8B427EF14F003018351320A70
:1027A000D8B43AEF14F05CEF26F004014D0E826FBE
:1027B00073EC0EF079EC2DF084C331F185C332F166
:1027C00086C333F10101296B86EC2DF0FDEC2CF072
:1027D00003018351300AD8B4FCEF13F00301835195
:1027E000310AD8B404EF14F003018351320AD8B48B
:1027F0000CEF14F05CEF26F0FD0E0C6E00C10BF038
:102800000AEC0BF014EF14F0FE0E0C6E00C10BF08E
:102810000AEC0BF027EF14F0FF0E0C6E00C10BF06A
:102820000AEC0BF03AEF14F00401300E826F73ECF7
:102830000EF004012C0E826F73EC0EF038EC2DF0CC
:10284000FD0E21EC0BF0E8CF00F14BEF14F004018A
:10285000310E826F73EC0EF004012C0E826F73EC5C
:102860000EF038EC2DF0FE0E21EC0BF0E8CF00F16D
:102870004BEF14F00401320E826F73EC0EF038EC63
:102880002DF004012C0E826F73EC0EF0FF0E21EC84
:102890000BF0E8CF00F1DBEC2CF031C182F4040145
:1028A000300E822773EC0EF032C182F40401300E38
:1028B000822773EC0EF033C182F40401300E8227BC
:1028C00073EC0EF05AEF26F003018351300AD8B4AE
:1028D0005FEF19F003018351310AD8B48CEF1AF07D
:1028E00003018351320AD8B4FAEF1AF0030183517D
:1028F000330AD8B40AEF1BF003018351340AD8B469
:102900001AEF1BF003018351350AD8B4A0EF1CF075
:1029100003018351360AD8B4CEEF1CF00301835172
:10292000370AD8B437EF17F003018351380AD8B407
:10293000D5EF17F003018351460AD8B4F3EF1BF02B
:10294000030183514D0AD8B4B0EF15F00301835150
:102950006D0AD8B4CAEF15F0030183515A0AD8B4EE
:1029600006EF1AF003018351490AD8B4CEEF1DF0E7
:1029700003018351500AD8B400EF1DF003018351C5
:10298000540AD8B479EF1DF003018351630AD8B417
:10299000EAEF15F003018351430AD8B4E2EF16F0D1
:1029A00003018351730AD8B4E8EF15F00301835192
:1029B000610AD8B4FDEF14F003018351650AD8B45D
:1029C000AFEF19F003018351450AD8B4BDEF19F0F8
:1029D00003018351620AD8B4CBEF19F0030183518C
:1029E000420AD8B4D9EF19F003018351760AD8B45A
:1029F000E7EF19F0D8A45CEF26F004014C0E826FCB
:102A000073EC0EF00401610E826F73EC0EF068EC53
:102A10002EF004012C0E826F73EC0EF038EC2DF0CA
:102A2000AFC500F10101DBEC2CF031C182F40401EF
:102A3000300E822773EC0EF032C182F40401300EA6
:102A4000822773EC0EF033C182F40401300E82272A
:102A500073EC0EF004012C0E826F73EC0EF038EC68
:102A60002DF0B0C500F10101DBEC2CF031C182F496
:102A70000401300E822773EC0EF032C182F404019F
:102A8000300E822773EC0EF033C182F40401300E55
:102A9000822773EC0EF004012C0E826F73EC0EF0A3
:102AA00038EC2DF0B1C500F10101DBEC2CF031C1A7
:102AB00082F40401300E822773EC0EF032C182F4EE
:102AC0000401300E822773EC0EF033C182F404014E
:102AD000300E822773EC0EF004012C0E826F73EC23
:102AE0000EF038EC2DF0B2C500F10101DBEC2CF05A
:102AF00031C182F40401300E822773EC0EF032C132
:102B000082F40401300E822773EC0EF033C182F49C
:102B10000401300E822773EC0EF004012C0E826F3C
:102B200073EC0EF038EC2DF0B6C500F10101DBECD2
:102B30002CF031C182F40401300E822773EC0EF0C8
:102B400032C182F40401300E822773EC0EF033C1DF
:102B500082F40401300E822773EC0EF0FCEF1CF0BF
:102B600079EC2DF084C333F186EC2DF0FDEC2CF0E4
:102B7000200E0C6E00C10BF00AEC0BF000C12FF51B
:102B800005012F51000A06E005012F51010A02E05C
:102B900002EC2FF004014C0E826F73EC0EF0040176
:102BA0004D0E826F73EC0EF004012C0E826F73ECED
:102BB0000EF038EC2DF02FC500F1DBEC2CF033C11A
:102BC00082F40401300E822773EC0EF0FCEF1CF04F
:102BD000F8EF33F004014C0E826F73EC0EF0040139
:102BE000630E826F73EC0EF0C0EC2DF004012C0E1E
:102BF000826F73EC0EF0FFEC15F0FCEF1CF038EC7C
:102C00002DF0B5C500F10101003B0F0E0017DBEC04
:102C10002CF033C182F40401300E822773EC0EF0E5
:102C2000B5C500F101010F0E01010017DBEC2CF01E
:102C300033C182F40401300E822773EC0EF00401DC
:102C40002D0E826F73EC0EF0B4C500F10101003B54
:102C50000F0E0017DBEC2CF033C182F40401300EB0
:102C6000822773EC0EF0B4C500F101010F0E0101D3
:102C70000017DBEC2CF033C182F40401300E822704
:102C800073EC0EF004012D0E826F73EC0EF0B3C5E1
:102C900000F10101003B0F0E0017DBEC2CF033C1FB
:102CA00082F40401300E822773EC0EF0B3C500F1FC
:102CB00001010F0E01010017DBEC2CF033C182F48F
:102CC0000401300E822773EC0EF00401200E826F97
:102CD00073EC0EF0B2C500F10F0E01010017DBEC32
:102CE0002CF033C182F40401300E822773EC0EF015
:102CF0000401200E826F73EC0EF0B1C500F10101EA
:102D00000101003B0F0E0017DBEC2CF033C182F405
:102D10000401300E822773EC0EF0B1C500F1010101
:102D20000F0E01010017DBEC2CF033C182F404011B
:102D3000300E822773EC0EF004013A0E826F73ECB2
:102D40000EF0B0C500F10101003B0F0E0017DBECE7
:102D50002CF033C182F40401300E822773EC0EF0A4
:102D6000B0C500F101010F0E01010017DBEC2CF0E2
:102D700033C182F40401300E822773EC0EF004019B
:102D80003A0E826F73EC0EF0AFC500F10101003B0B
:102D90000F0E0017DBEC2CF033C182F40401300E6F
:102DA000822773EC0EF0AFC500F101010F0E001782
:102DB000DBEC2CF033C182F40401300E822773EC7B
:102DC0000EF0120084C3E8FF0F0BE83AE8CFB5F528
:102DD00085C3E8FF0F0B0501B51387C3E8FF0F0B91
:102DE000E83AE8CFB4F588C3E8FF0F0B0501B41348
:102DF0008AC3E8FF0F0BE83AE8CFB3F58BC3E8FFCF
:102E00000F0B0501B3138DC3E8FF0F0BE8CFB2F52D
:102E10008FC3E8FF0F0BE83AE8CFB1F590C3E8FFA6
:102E20000F0B0501B11392C3E8FF0F0BE83AE8CF8F
:102E3000B0F593C3E8FF0F0B0501B01395C3E8FF8E
:102E40000F0BE83AE8CFAFF596C3E8FF0F0B05018B
:102E5000AF131BEC2EF004014C0E826F73EC0EF0DE
:102E60000401430E826F73EC0EF0F4EF15F007844B
:102E700004014C0E826F73EC0EF00401370E826F6A
:102E800073EC0EF004012C0E826F73EC0EF0050152
:102E90002E51130A06E005012E51170A0DE0D2EF5C
:102EA00017F00101000E006F000E016F100E026F8F
:102EB000000E036F65EF17F00101000E006F000EAA
:102EC000016F000E026F010E036FDBEC2CF02AC1C4
:102ED00082F40401300E822773EC0EF02BC182F4D1
:102EE0000401300E822773EC0EF02CC182F4040131
:102EF000300E822773EC0EF02DC182F40401300EE7
:102F0000822773EC0EF02EC182F40401300E82276A
:102F100073EC0EF02FC182F40401300E822773ECA3
:102F20000EF030C182F40401300E822773EC0EF0F3
:102F300031C182F40401300E822773EC0EF032C1ED
:102F400082F40401300E822773EC0EF033C182F458
:102F50000401300E822773EC0EF004012C0E826FF8
:102F600073EC0EF00101100E006F000E016F000EE9
:102F7000026F000E036FDBEC2CF031C182F4040110
:102F8000300E822773EC0EF032C182F40401300E51
:102F9000822773EC0EF033C182F40401300E8227D5
:102FA00073EC0EF00794FCEF1CF00501216B226B13
:102FB000236B246B04014C0E826F73EC0EF0040142
:102FC000380E826F73EC0EF004012C0E826F73ECDE
:102FD0000EF00101100E006F000E016F000E026F67
:102FE000000E036FDBEC2CF02AC182F40401300EDA
:102FF000822773EC0EF02BC182F40401300E82277D
:1030000073EC0EF02CC182F40401300E822773ECB5
:103010000EF02DC182F40401300E822773EC0EF005
:103020002EC182F40401300E822773EC0EF02FC102
:1030300082F40401300E822773EC0EF030C182F46A
:103040000401300E822773EC0EF031C182F40401CA
:10305000300E822773EC0EF032C182F40401300E80
:10306000822773EC0EF033C182F40401300E822704
:1030700073EC0EF004012C0E826F73EC0EF025C57C
:1030800000F126C501F127C502F128C503F10101B0
:10309000100E046F000E056F000E066F000E076F16
:1030A0006EEC2CF000C133F501C134F502C135F5E9
:1030B00003C136F5DBEC2CF02AC182F40401300E9A
:1030C000822773EC0EF02BC182F40401300E8227AC
:1030D00073EC0EF02CC182F40401300E822773ECE5
:1030E0000EF02DC182F40401300E822773EC0EF035
:1030F0002EC182F40401300E822773EC0EF02FC132
:1031000082F40401300E822773EC0EF030C182F499
:103110000401300E822773EC0EF031C182F40401F9
:10312000300E822773EC0EF032C182F40401300EAF
:10313000822773EC0EF033C182F40401300E822733
:1031400073EC0EF07DEC0EF005013367AFEF18F075
:103150003467AFEF18F03567AFEF18F0366702D07D
:103160004EEF19F0129E129C21C500F122C501F10B
:1031700023C502F124C503F1899A400EC76E200EC3
:10318000C66E9E96C69E0B0EC96EFF0E9EB602D0F0
:10319000E82EFCD79E96C69E02C1C9FFFF0E9EB6C2
:1031A00002D0E82EFCD79E96C69E01C1C9FFFF0E35
:1031B0009EB602D0E82EFCD79E96C69E00C1C9FFDF
:1031C000FF0E9EB602D0E82EFCD79E96C69EC95230
:1031D000FF0E9EB602D0E82EFCD70501100E326F0E
:1031E000040114EE00F080517F0BE1269E96C69EEE
:1031F000C952FF0E9EB602D0E82EFCD7C9CFE7FF1A
:103200000401802B0501322FF0EF18F0898A33C5B5
:1032100000F134C501F135C502F136C503F10101F4
:10322000010E046F000E056F000E066F000E076F93
:103230003DEC2CF000C133F501C134F502C135F588
:1032400003C136F5050133672DEF19F034672DEF13
:1032500019F035672DEF19F0366702D04EEF19F0EF
:1032600021C500F122C501F123C502F124C503F1F6
:103270000101100E046F000E056F000E066F000EA8
:10328000076F42EC2CF000C121F501C122F502C10B
:1032900023F503C124F5128E5CEF26F00401450EE0
:1032A000826F73EC0EF004014F0E826F73EC0EF020
:1032B0000401460E826F73EC0EF0FCEF1CF00784E5
:1032C000B9EC33F038EC2DF02DC500F1DBEC2CF02F
:1032D00004014C0E826F73EC0EF00401300E826F0D
:1032E00073EC0EF004012C0E826F73EC0EF031C102
:1032F00082F40401300E822773EC0EF032C182F4A6
:103300000401300E822773EC0EF033C182F4040105
:10331000300E822773EC0EF004012C0E826F73ECDA
:103320000EF038EC2DF02EC500F1DBEC2CF031C1A5
:1033300082F40401300E822773EC0EF032C182F465
:103340000401300E822773EC0EF033C182F40401C5
:10335000300E822773EC0EF00794FCEF1CF0040192
:103360004C0E826F73EC0EF00401650E826F73ECED
:103370000EF0DEEC2FF0FCEF1CF004014C0E826F1F
:1033800073EC0EF00401450E826F73EC0EF0F5EC59
:103390002FF0FCEF1CF004014C0E826F73EC0EF06A
:1033A0000401620E826F73EC0EF023EC30F0FCEF40
:1033B0001CF004014C0E826F73EC0EF00401420EFF
:1033C000826F73EC0EF00CEC30F0FCEF1CF004019B
:1033D0004C0E826F73EC0EF00401760E826F73EC6C
:1033E0000EF004012C0E826F73EC0EF010A807D0C3
:1033F0000401310E826F73EC0EF0FCEF1CF004013F
:10340000300E826F73EC0EF0FCEF1CF004014C0EDA
:10341000826F73EC0EF004015A0E826F73EC0EF0A3
:1034200004012C0E826F73EC0EF0B9EC33F038EC23
:103430002DF005012E51130A06E005012E51170A41
:103440000DE037EF1AF00101000E006F000E016F62
:10345000100E026F000E036F37EF1AF00101000E1D
:10346000006F000E016F000E026F010E036F01016D
:10347000100E046F000E056F000E066F000E076F32
:103480006EEC2CF0DBEC2CF02AC182F40401300E3F
:10349000822773EC0EF02BC182F40401300E8227D8
:1034A00073EC0EF02CC182F40401300E822773EC11
:1034B0000EF02DC182F40401300E822773EC0EF061
:1034C0002EC182F40401300E822773EC0EF02FC15E
:1034D00082F40401300E822773EC0EF030C182F4C6
:1034E0000401300E822773EC0EF031C182F4040126
:1034F000300E822773EC0EF032C182F40401300EDC
:10350000822773EC0EF033C182F40401300E82275F
:1035100073EC0EF0FCEF1CF0078404014C0E826F7C
:1035200073EC0EF00401310E826F73EC0EF00401A7
:103530002C0E826F73EC0EF025C500F126C501F14B
:1035400027C502F128C503F10101100E046F000E1A
:10355000056F000E066F000E076F6EEC2CF0DBECB3
:103560002CF02AC182F40401300E822773EC0EF095
:103570002BC182F40401300E822773EC0EF02CC1B3
:1035800082F40401300E822773EC0EF02DC182F418
:103590000401300E822773EC0EF02EC182F4040178
:1035A000300E822773EC0EF02FC182F40401300E2E
:1035B000822773EC0EF030C182F40401300E8227B2
:1035C00073EC0EF031C182F40401300E822773ECEB
:1035D0000EF032C182F40401300E822773EC0EF03B
:1035E00033C182F40401300E822773EC0EF007948D
:1035F000FCEF1CF0078404014C0E826F73EC0EF09C
:103600000401320E826F73EC0EF011EC32F007946D
:10361000FCEF1CF0078404014C0E826F73EC0EF07B
:103620000401330E826F73EC0EF06EEC32F00794EF
:1036300097EF1AF0078404014C0E826F73EC0EF0C2
:103640000401340E826F73EC0EF004012C0E826FB5
:1036500073EC0EF079EC2DF084C32AF185C32BF1C5
:1036600086C32CF187C32DF188C32EF189C32FF1B6
:103670008AC330F18BC331F18CC332F18DC333F186
:103680000101296B86EC2DF0FDEC2CF0100E046F7F
:10369000000E056F000E066F000E076F4EEC2CF04B
:1036A00000C121F501C122F502C123F503C124F5B2
:1036B0006CEC33F038C5AFF539C5B0F53AC5B1F5A6
:1036C0003BC5B2F53CC5B3F53DC5B4F53EC5B5F552
:1036D000FFEC15F004012C0E826F73EC0EF03FC569
:1036E00000F140C501F141C502F142C503F10101FC
:1036F000000E046F000E056F010E066F000E076FBF
:103700006EEC2CF0DBEC2CF0296789EF1BF08EEFD0
:103710001BF004012D0E826F73EC0EF030C182F4A9
:103720000401300E822773EC0EF031C182F40401E3
:10373000300E822773EC0EF004012E0E826F73ECB4
:103740000EF032C182F40401300E822773EC0EF0C9
:1037500033C182F40401300E822773EC0EF00401B1
:103760002C0E826F73EC0EF038EC2DF043C500F197
:1037700044C501F186EC27F004012C0E826F73EC36
:103780000EF038EC2DF045C500F1DBEC2CF031C12A
:1037900082F40401300E822773EC0EF032C182F401
:1037A0000401300E822773EC0EF033C182F4040161
:1037B000300E822773EC0EF004012C0E826F73EC36
:1037C0000EF037C5E8FFE8B806D00401300E826F6E
:1037D00073EC0EF005D00401310E826F73EC0EF025
:1037E0000794FCEF1CF079EC2DF085C32AF186C319
:1037F0002BF187C32CF188C32DF189C32EF18AC325
:103800002FF18BC330F18CC331F18DC332F18EC3F4
:1038100033F10101296B86EC2DF0FDEC2CF0010158
:10382000010E046F000E056F000E066F000E076F8D
:103830003DEC2CF0100E046F000E056F000E066FAD
:10384000000E076F4EEC2CF000C129F501C12AF5DE
:1038500002C12BF503C12CF598EC31F004014C0E9C
:10386000826F73EC0EF00401460E826F73EC0EF063
:1038700004012C0E826F73EC0EF025C500F126C5F5
:1038800001F127C502F128C503F10101100E046FF3
:10389000000E056F000E066F000E076F6EEC2CF029
:1038A000DBEC2CF02AC182F40401300E822773EC89
:1038B0000EF02BC182F40401300E822773EC0EF05F
:1038C0002CC182F40401300E822773EC0EF02DC15E
:1038D00082F40401300E822773EC0EF02EC182F4C4
:1038E0000401300E822773EC0EF02FC182F4040124
:1038F000300E822773EC0EF030C182F40401300EDA
:10390000822773EC0EF031C182F40401300E82275D
:1039100073EC0EF032C182F40401300E822773EC96
:103920000EF033C182F40401300E822773EC0EF0E6
:10393000FCEF1CF00F986EEC32F030805CEF26F05C
:1039400004014C0E826F73EC0EF00401350E826F91
:1039500073EC0EF004012C0E826F73EC0EF038EC59
:103960002DF00784B9C500F10794DBEC2CF031C1D0
:1039700082F40401300E822773EC0EF032C182F41F
:103980000401300E822773EC0EF033C182F404017F
:10399000300E822773EC0EF0FCEF1CF031EC32F0AD
:1039A00038EC2DF037C500F1DBEC2CF004014C0EA7
:1039B000826F73EC0EF00401360E826F73EC0EF022
:1039C00004012C0E826F73EC0EF031C182F40401FD
:1039D000300E822773EC0EF032C182F40401300EF7
:1039E000822773EC0EF033C182F40401300E82277B
:1039F00073EC0EF0FCEF1CF07DEC0EF05CEF26F0AB
:103A000004014C0E826F73EC0EF00401500E826FB5
:103A100073EC0EF004012C0E826F73EC0EF085C374
:103A20002AF186C32BF187C32CF188C32DF189C3FA
:103A30002EF18AC32FF18BC330F18CC331F18DC3CA
:103A400032F18EC333F1010186EC2DF0FDEC2CF048
:103A500003018451530A0DE0030184514D0A38E0FB
:103A60000401780E826F73EC0EF07DEC0EF05CEFCB
:103A700026F00401530E826F73EC0EF0250E0C6ECF
:103A800000C10BF00AEC0BF0260E0C6E01C10BF01E
:103A90000AEC0BF0270E0C6E02C10BF00AEC0BF0D7
:103AA000280E0C6E03C10BF00AEC0BF000C157F5A9
:103AB00001C158F502C159F503C15AF500C15BF5C2
:103AC00001C15CF502C15DF503C15EF5DDEF1DF0DE
:103AD00004014D0E826F73EC0EF0290E0C6E00C1C6
:103AE0000BF00AEC0BF000C15FF500C160F5DDEFF3
:103AF0001DF004014C0E826F73EC0EF00401540EA5
:103B0000826F73EC0EF004012C0E826F73EC0EF0DA
:103B100084C32AF185C32BF186C32CF187C32DF111
:103B200088C32EF189C32FF18AC330F18BC331F1E1
:103B30008DC332F18EC333F1010186EC2DF0FDEC23
:103B40002CF00101000E046F000E056F010E066FD0
:103B5000000E076F4EEC2CF0210E0C6E00C10BF026
:103B60000AEC0BF0220E0C6E01C10BF00AEC0BF00C
:103B7000230E0C6E02C10BF00AEC0BF0240E0C6E3F
:103B800003C10BF00AEC0BF000C161F501C162F555
:103B900002C163F503C164F5DDEF1DF004014C0EB5
:103BA000826F73EC0EF00401490E826F73EC0EF01D
:103BB00004012C0E826F73EC0EF0250E21EC0BF03D
:103BC000E8CF00F1260E21EC0BF0E8CF01F1270E33
:103BD00021EC0BF0E8CF02F1280E21EC0BF0E8CF3E
:103BE00003F1DBEC2CF09EEC2AF00401730E826FE3
:103BF00073EC0EF004012C0E826F73EC0EF038ECB7
:103C00002DF0290E21EC0BF0E8CF00F1DBEC2CF0CD
:103C10009EEC2AF004016D0E826F73EC0EF004012D
:103C20002C0E826F73EC0EF05BC500F15CC501F1E8
:103C30005DC502F15EC503F1DBEC2CF09EEC2AF0D1
:103C40000401730E826F73EC0EF004012C0E826F70
:103C500073EC0EF038EC2DF060C500F1DBEC2CF0CD
:103C60009EEC2AF004016D0E826F73EC0EF00401DD
:103C70002C0E826F73EC0EF061C500F162C501F18C
:103C800063C502F164C503F177EC26F004012C0E44
:103C9000826F73EC0EF07DEC0EF05CEF26F083C3C8
:103CA0002AF184C32BF185C32CF186C32DF187C380
:103CB0002EF188C32FF189C330F18AC331F18BC350
:103CC00032F18CC333F1010186EC2DF0FDEC2CF0C8
:103CD000160E0C6E00C10BF00AEC0BF0170E0C6EFA
:103CE00001C10BF00AEC0BF0180E0C6E02C10BF0C8
:103CF0000AEC0BF0190E0C6E03C10BF00AEC0BF082
:103D000000C18AF101C18BF102C18CF103C18DF1B7
:103D100000C18EF101C18FF102C190F103C191F197
:103D200031EF1FF083C32AF184C32BF185C32CF13B
:103D300086C32DF187C32EF188C32FF189C330F1DB
:103D40008AC331F18BC332F18CC333F1010186ECAC
:103D50002DF0FDEC2CF000C18AF101C18BF102C104
:103D60008CF103C18DF100C18EF101C18FF102C14F
:103D700090F103C191F131EF1FF083C32AF184C3A5
:103D80002BF185C32CF186C32DF187C32EF188C397
:103D90002FF189C330F18AC331F18CC332F18DC365
:103DA00033F1010186EC2DF0FDEC2CF00101000E49
:103DB000046F000E056F010E066F000E076F4EECCC
:103DC0002CF01A0E0C6E00C10BF00AEC0BF01B0E5F
:103DD0000C6E01C10BF00AEC0BF01C0E0C6E02C154
:103DE0000BF00AEC0BF01D0E0C6E03C10BF00AEC8D
:103DF0000BF000C192F101C193F102C194F103C132
:103E000095F131EF1FF083C32AF184C32BF185C3F1
:103E10002CF186C32DF187C32EF188C32FF189C3FE
:103E200030F18AC331F18CC332F18DC333F101011A
:103E300086EC2DF0FDEC2CF00101000E046F000E5D
:103E4000056F010E066F000E076F4EEC2CF000C1DF
:103E500092F101C193F102C194F103C195F131EFE7
:103E60001FF0160E21EC0BF0E8CF00F1170E21EC3D
:103E70000BF0E8CF01F1180E21EC0BF0E8CF02F1C6
:103E8000190E21EC0BF0E8CF03F1DBEC2CF09EECEB
:103E90002AF00401730E826F73EC0EF004012C0EF5
:103EA000826F73EC0EF08AC100F18BC101F18CC1FD
:103EB00002F18DC103F1DBEC2CF09EEC2AF0040141
:103EC000730E826F73EC0EF004012C0E826F73EC94
:103ED0000EF01A0E21EC0BF0E8CF00F11B0E21ECD6
:103EE0000BF0E8CF01F11C0E21EC0BF0E8CF02F152
:103EF0001D0E21EC0BF0E8CF03F177EC26F0040166
:103F00002C0E826F73EC0EF092C100F193C101F19F
:103F100094C102F195C103F177EC26F07DEC0EF02F
:103F20005CEF26F00401690E826F73EC0EF0040161
:103F30002C0E826F73EC0EF00101040E006F000E68
:103F4000016F000E026F000E036FDBEC2CF02CC132
:103F500082F40401300E822773EC0EF02DC182F43E
:103F60000401300E822773EC0EF02EC182F404019E
:103F7000300E822773EC0EF02FC182F40401300E54
:103F8000822773EC0EF030C182F40401300E8227D8
:103F900073EC0EF031C182F40401300E822773EC11
:103FA0000EF032C182F40401300E822773EC0EF061
:103FB00033C182F40401300E822773EC0EF0040149
:103FC0002C0E826F73EC0EF00101060E006F000ED6
:103FD000016F000E026F000E036FDBEC2CF02CC1A2
:103FE00082F40401300E822773EC0EF02DC182F4AE
:103FF0000401300E822773EC0EF02EC182F404010E
:10400000300E822773EC0EF02FC182F40401300EC3
:10401000822773EC0EF030C182F40401300E822747
:1040200073EC0EF031C182F40401300E822773EC80
:104030000EF032C182F40401300E822773EC0EF0D0
:1040400033C182F40401300E822773EC0EF00401B8
:104050002C0E826F73EC0EF00101390E006F000E12
:10406000016F000E026F000E036FDBEC2CF02CC111
:1040700082F40401300E822773EC0EF02DC182F41D
:104080000401300E822773EC0EF02EC182F404017D
:10409000300E822773EC0EF02FC182F40401300E33
:1040A000822773EC0EF030C182F40401300E8227B7
:1040B00073EC0EF031C182F40401300E822773ECF0
:1040C0000EF032C182F40401300E822773EC0EF040
:1040D00033C182F40401300E822773EC0EF0040128
:1040E0002C0E826F73EC0EF0200EF86EF76AF66AF3
:1040F00004010900F5CF82F473EC0EF00900F5CF4E
:1041000082F473EC0EF00900F5CF82F473EC0EF03C
:104110000900F5CF82F473EC0EF00900F5CF82F4BC
:1041200073EC0EF00900F5CF82F473EC0EF0090089
:10413000F5CF82F473EC0EF00900F5CF82F473EC46
:104140000EF07DEC0EF05CEF26F08351630AD8A4EC
:104150005AEF26F08451610AD8A45AEF26F085510F
:104160006C0AD8A45AEF26F08651410A3FE08651E6
:10417000440A1BE08651420AD8B409EF21F0865167
:10418000350AD8B4E6EF27F08651360AD8B43BEFAB
:1041900028F08651370AD8B4A4EF28F08651380A9F
:1041A000D8B402EF29F05AEF26F00798079A0401D5
:1041B0007A0E826F73EC0EF00401780E826F73EC4E
:1041C0000EF00401640E826F73EC0EF00401550EC4
:1041D000826F73EC0EF0F2EF20F004014C0E826F50
:1041E00073EC0EF07DEC0EF05CEF26F00788079A7A
:1041F00004017A0E826F73EC0EF00401410E826F9F
:1042000073EC0EF00401610E826F73EC0EF0E6EFBA
:1042100020F00798078A04017A0E826F73EC0EF083
:104220000401420E826F73EC0EF00401610E826F86
:1042300073EC0EF0E6EF20F00101666727EF21F046
:10424000676727EF21F0686727EF21F0696715D0CE
:104250004F6732EF21F0506732EF21F0516732EFB4
:1042600021F052670AD00101000E006F000E016FAD
:10427000000E026F000E036F120011B80AD0010188
:10428000620E046F010E056F000E066F000E076FC1
:1042900009D00101A70E046F020E056F000E066F14
:1042A000000E076F66C100F167C101F168C102F13C
:1042B00069C103F13DEC2CF003BFCFEF21F0119A5F
:1042C000119C0101000E046FA80E056F550E066FBC
:1042D000020E076F66C100F167C101F168C102F10A
:1042E00069C103F166C186F167C187F168C188F1D0
:1042F00069C189F13DEC2CF003BF0BD00101000E28
:10430000866FA80E876F550E886F020E896F118A0F
:10431000119C0E0E21EC0BF0E8CF18F10F0E21ECE2
:104320000BF0E8CF19F1100E21EC0BF0E8CF1AF1E9
:10433000110E21EC0BF0E8CF1BF186EC2BF086C1BF
:1043400004F187C105F188C106F189C107F13DEC8F
:104350002CF007824AEC2BF086EC2BF007924AEC0B
:104360002BF086C100F187C101F188C102F189C13A
:1043700003F107924AEC2BF0CC0E046FE00E056FB0
:10438000870E066F050E076F3DEC2CF000C118F18B
:1043900001C119F102C11AF103C11BF13BD0119CFB
:1043A000119A0101800E006F1A0E016F060E026F46
:1043B000000E036F4FC104F150C105F151C106F168
:1043C00052C107F13DEC2CF003AF05D038EC2DF0D5
:1043D000118C119A12000E0E21EC0BF0E8CF18F19F
:1043E0000F0E21EC0BF0E8CF19F1100E21EC0BF0C1
:1043F000E8CF1AF1110E21EC0BF0E8CF1BF14FC101
:1044000000F150C101F151C102F152C103F1078223
:104410004AEC2BF018C100F119C101F11AC102F1E7
:104420001BC103F112000401730E826F73EC0EF0D6
:1044300004012C0E826F73EC0EF0078462C166F1EA
:1044400063C167F164C168F165C169F14BC14FF1A6
:104450004CC150F14DC151F14EC152F157C159F10A
:1044600058C15AF1079439EC22F07DEC0EF05CEF64
:1044700026F066C100F167C101F168C102F169C1AE
:1044800003F10101DBEC2CF09EEC2AF00401630E39
:10449000826F73EC0EF004012C0E826F73EC0EF041
:1044A0004FC100F150C101F151C102F152C103F1FC
:1044B0000101DBEC2CF09EEC2AF00401660E826F09
:1044C00073EC0EF004012C0E826F73EC0EF038ECDE
:1044D0002DF059C100F15AC101F10101DBEC2CF0C2
:1044E0009EEC2AF00401740E826F73EC0EF0120041
:1044F00010820401530E826F73EC0EF004012C0E37
:10450000826F73EC0EF083C32AF184C32BF185C351
:104510002CF186C32DF187C32EF188C32FF189C3F7
:1045200030F18AC331F18BC332F18CC333F1010115
:1045300086EC2DF0FDEC2CF000C166F101C167F1B5
:1045400002C168F103C169F18EC32AF18FC32BF157
:1045500090C32CF191C32DF192C32EF193C32FF18F
:1045600094C330F195C331F196C332F197C333F15F
:10457000010186EC2DF0FDEC2CF000C14FF101C1E2
:1045800050F102C151F103C152F179EC2DF099C300
:104590002FF19AC330F19BC331F19CC332F19DC31B
:1045A00033F1010186EC2DF0FDEC2CF000C159F146
:1045B00001C15AF139EC22F004012C0E826F73EC28
:1045C0000EF0F3EF22F0118E19A002D019AE108C6C
:1045D00018BE02D018A4108E03018251520A02E1C3
:1045E0000F8201D00F928251750A02E1108401D02E
:1045F00010948251550A02E1108601D0109611A044
:1046000003D011A401D01084078410B261EF23F00D
:1046100010A44DEF23F0B6C166F1B7C167F1B8C180
:1046200068F1B9C169F1BAC16AF1BBC16BF1BCC132
:104630006CF1BDC16DF1BEC16EF1BFC16FF1C0C102
:1046400070F1C1C171F1C2C172F1C3C173F1C4C1D2
:1046500074F1C5C175F1C6C176F1C7C177F1C8C1A2
:1046600078F1C9C179F1CAC17AF1CBC17BF1CCC172
:104670007CF1CDC17DF1CEC17EF1CFC17FF1D0C142
:1046800080F1D1C181F1D2C182F1D3C183F1D4C112
:1046900084F1D5C185F155EF23F062C166F163C1A4
:1046A00067F164C168F165C169F14BC14FF14CC15B
:1046B00050F14DC151F14EC152F157C159F158C19C
:1046C0005AF107940FA083EF23F00101926770EF76
:1046D00023F0936770EF23F0946770EF23F09567F2
:1046E00074EF23F083EF23F01CEC21F092C104F16E
:1046F00093C105F194C106F195C107F13DEC2CF091
:1047000003BF20EF26F01CEC21F00101000E046F26
:10471000000E056F010E066F000E076F6EEC2CF099
:1047200011A02AD011A228D0DBEC2CF0296701D0EF
:1047300005D004012D0E826F73EC0EF030C182F4AF
:104740000401300E822773EC0EF031C182F40401B3
:10475000300E822773EC0EF032C182F40401300E69
:10476000822773EC0EF033C182F40401300E8227ED
:1047700073EC0EF07DEC0EF012A8C5D012981AC0A2
:104780001BF01B3A1B42070E1B1600011B50000AB0
:10479000D8B44FEF24F000011B50010AD8B4DBEF6E
:1047A00023F000011B50020AD8B4D9EF23F081EFA7
:1047B00024F081EF24F038EC2DF02AC001F12BC059
:1047C00000F1D89001330033D89001330033010158
:1047D000630E046F000E056F000E066F000E076F6C
:1047E0006EEC2CF0280E046F000E056F000E066FA5
:1047F000000E076F3DEC2CF000C12DF038EC2DF0D1
:1048000028C001F1019F019D29C000F10101A40E02
:10481000046F000E056F000E066F000E076F6EEC42
:104820002CF000C12CF000C104F101C105F102C15E
:1048300006F103C107F1640E006F000E016F000E58
:10484000026F000E036F3DEC2CF0050E046F000E9E
:10485000056F000E066F000E076F6EEC2CF000C1A6
:1048600004F101C105F102C106F103C107F138EC01
:104870002DF02DC000F13DEC2CF000C12EF02EC02B
:10488000E8FF050F2D5C03E78A8481EF24F02EC03A
:10489000E8FF0A0F2D5C01E68A9481EF24F000C145
:1048A00024F101C125F102C126F103C127F138EC41
:1048B0002DF03EEC2DF01A501F0BE8CF00F1010156
:1048C000640E046F000E056F000E066F000E076F7A
:1048D0004EEC2CF024C104F125C105F126C106F1EE
:1048E00027C107F13DEC2CF003BF02D08A9401D020
:1048F0008A8424C100F125C101F126C102F127C13A
:1049000003F15CEF26F000C124F101C125F102C1E1
:1049100026F103C127F110AE4DD0109E00C108F161
:1049200001C109F102C10AF103C10BF1DBEC2CF06A
:1049300030C1D6F131C1D7F132C1D8F133C1D9F18B
:1049400008C100F109C101F10AC102F10BC103F173
:1049500001016C0E046F070E056F000E066F000E4E
:10496000076F3DEC2CF003BF04D00101550EDA6F48
:104970001CD008C100F109C101F10AC102F10BC14B
:1049800003F10101A40E046F060E056F000E066F01
:10499000000E076F3DEC2CF003BF04D001017F0E29
:1049A000DA6F03D00101FF0EDA6F1C8E11AE20EF1B
:1049B00026F0119E24C100F125C101F126C102F1AA
:1049C00027C103F111A005D011A203D00FB020EF31
:1049D00026F010A4F3EF24F00401750E826F73EC3F
:1049E0000EF0F8EF24F00401720E826F73EC0EF0FB
:1049F00004012C0E826F73EC0EF0DBEC2CF02967B7
:104A000007EF25F00401200E826F0AEF25F0040164
:104A10002D0E826F73EC0EF030C182F40401300E63
:104A2000822773EC0EF031C182F40401300E82272C
:104A300073EC0EF004012E0E826F73EC0EF032C197
:104A400082F40401300E822773EC0EF033C182F43D
:104A50000401300E822773EC0EF004016D0E826F9C
:104A600073EC0EF004012C0E826F73EC0EF04FC14C
:104A700000F150C101F151C102F152C103F1010134
:104A8000DBEC2CF09EEC2AF00401480E826F73ECF4
:104A90000EF004017A0E826F73EC0EF004012C0EFE
:104AA000826F73EC0EF066C100F167C101F168C15D
:104AB00002F169C103F10101DBEC2CF09EEC2AF05C
:104AC0000401630E826F73EC0EF004012C0E826FF2
:104AD00073EC0EF066C100F167C101F168C102F12B
:104AE00069C103F101010A0E046F000E056F000E8B
:104AF000066F000E076F4EEC2CF0000E046F120EC6
:104B0000056F000E066F000E076F6EEC2CF0DBECED
:104B10002CF02AC182F40401300E822773EC0EF0CF
:104B20002BC182F40401300E822773EC0EF02CC1ED
:104B300082F40401300E822773EC0EF02DC182F452
:104B40000401300E822773EC0EF02EC182F40401B2
:104B5000300E822773EC0EF02FC182F40401300E68
:104B6000822773EC0EF030C182F40401300E8227EC
:104B700073EC0EF004012E0E826F73EC0EF031C157
:104B800082F40401300E822773EC0EF032C182F4FD
:104B90000401300E822773EC0EF033C182F404015D
:104BA000300E822773EC0EF00401730E826F73ECEB
:104BB0000EF004012C0E826F73EC0EF038EC2DF029
:104BC00059C100F15AC101F186EC27F00FB2ECEFA8
:104BD00025F00FA01EEF26F004012C0E826F73EC5F
:104BE0000EF0200EF86EF76AF66A04010900F5CFA0
:104BF00082F473EC0EF00900F5CF82F473EC0EF042
:104C00000900F5CF82F473EC0EF00900F5CF82F4C1
:104C100073EC0EF00900F5CF82F473EC0EF009008E
:104C2000F5CF82F473EC0EF00900F5CF82F473EC4B
:104C30000EF00900F5CF82F473EC0EF07DEC0EF06F
:104C40000F90109E12985CEF26F00401630E826FA5
:104C500073EC0EF004012C0E826F73EC0EF062EC1C
:104C600026F004012C0E826F73EC0EF0D5EC26F0CA
:104C700004012C0E826F73EC0EF051EC27F004014E
:104C80002C0E826F73EC0EF00101F80E006FCD0E4A
:104C9000016F660E026F030E036F77EC26F00401BE
:104CA0002C0E826F73EC0EF067EC27F07DEC0EF0AB
:104CB0005CEF26F07DEC0EF00301C26B07901092C2
:104CC0006BEF29F0D8900E0E21EC0BF0E8CF00F13D
:104CD0000F0E21EC0BF0E8CF01F1100E21EC0BF0E0
:104CE000E8CF02F1110E21EC0BF0E8CF03F1010146
:104CF000000E046F000E056F010E066F000E076FA9
:104D00006EEC2CF0DBEC2CF02AC182F40401300EA6
:104D1000822773EC0EF02BC182F40401300E82273F
:104D200073EC0EF02CC182F40401300E822773EC78
:104D30000EF02DC182F40401300E822773EC0EF0C8
:104D40002EC182F40401300E822773EC0EF02FC1C5
:104D500082F40401300E822773EC0EF030C182F42D
:104D60000401300E822773EC0EF031C182F404018D
:104D7000300E822773EC0EF004012E0E826F73EC5E
:104D80000EF032C182F40401300E822773EC0EF073
:104D900033C182F40401300E822773EC0EF004015B
:104DA0006D0E826F73EC0EF01200120E21EC0BF000
:104DB000E8CF00F1130E21EC0BF0E8CF01F1140E57
:104DC00021EC0BF0E8CF02F1150E21EC0BF0E8CF4F
:104DD00003F101010A0E046F000E056F000E066F4D
:104DE000000E076F4EEC2CF0000E046F120E056FD4
:104DF000000E066F000E076F6EEC2CF0DBEC2CF053
:104E00002AC182F40401300E822773EC0EF02BC10C
:104E100082F40401300E822773EC0EF02CC182F470
:104E20000401300E822773EC0EF02DC182F40401D0
:104E3000300E822773EC0EF02EC182F40401300E86
:104E4000822773EC0EF02FC182F40401300E82270A
:104E500073EC0EF030C182F40401300E822773EC43
:104E60000EF004012E0E826F73EC0EF031C182F44D
:104E70000401300E822773EC0EF032C182F404017B
:104E8000300E822773EC0EF033C182F40401300E31
:104E9000822773EC0EF00401730E826F73EC0EF038
:104EA00012000A0E21EC0BF0E8CF00F10B0E21EC02
:104EB0000BF0E8CF01F10C0E21EC0BF0E8CF02F182
:104EC0000D0E21EC0BF0E8CF03F186EF27F0060E74
:104ED00021EC0BF0E8CF00F1070E21EC0BF0E8CF4E
:104EE00001F1080E21EC0BF0E8CF02F1090E21ECE4
:104EF0000BF0E8CF03F186EF27F0010138EC2DF03D
:104F0000078457C100F158C101F107940101E80E6F
:104F1000046F800E056F000E066F000E076F4EECDB
:104F20002CF0000E046F040E056F000E066F000ECD
:104F3000076F6EEC2CF0880E046F130E056F000ED9
:104F4000066F000E076F3DEC2CF00A0E046F000E8A
:104F5000056F000E066F000E076F6EEC2CF0DBEC99
:104F60002CF001012967BAEF27F00401200E826FAF
:104F7000BDEF27F004012D0E826F73EC0EF030C1EF
:104F800082F40401300E822773EC0EF031C182F4FA
:104F90000401300E822773EC0EF032C182F404015A
:104FA000300E822773EC0EF004012E0E826F73EC2C
:104FB0000EF033C182F40401300E822773EC0EF040
:104FC0000401430E826F73EC0EF0120087C32AF1C6
:104FD00088C32BF189C32CF18AC32DF18BC32EF129
:104FE0008CC32FF18DC330F18EC331F190C332F1F8
:104FF00091C333F10101296B86EC2DF0FDEC2CF00F
:105000000101000E046F000E056F010E066F000E09
:10501000076F4EEC2CF00E0E0C6E00C10BF00AEC7C
:105020000BF00F0E0C6E01C10BF00AEC0BF0100E22
:105030000C6E02C10BF00AEC0BF0110E0C6E03C1EA
:105040000BF00AEC0BF004017A0E826F73EC0EF099
:1050500004012C0E826F73EC0EF00401350E826F8A
:1050600073EC0EF004012C0E826F73EC0EF062EC08
:1050700026F0F2EF20F087C32AF188C32BF189C311
:105080002CF18AC32DF18BC32EF18CC32FF18DC36C
:1050900030F18EC331F190C332F191C333F101018C
:1050A000296B86EC2DF0FDEC2CF0880E046F130EAE
:1050B000056F000E066F000E076F42EC2CF0000E1D
:1050C000046F040E056F000E066F000E076F4EECA6
:1050D0002CF00101E80E046F800E056F000E066FC4
:1050E000000E076F6EEC2CF00A0E0C6E00C10BF078
:1050F0000AEC0BF00B0E0C6E01C10BF00AEC0BF07E
:105100000C0E0C6E02C10BF00AEC0BF00D0E0C6EC7
:1051100003C10BF00AEC0BF004017A0E826F73EC02
:105120000EF004012C0E826F73EC0EF00401360EAB
:10513000826F73EC0EF004012C0E826F73EC0EF094
:1051400051EC27F0F2EF20F087C32AF188C32BF14E
:1051500089C32CF18AC32DF18BC32EF18CC32FF19F
:105160008DC330F18FC331F190C332F191C333F16C
:10517000010186EC2DF0FDEC2CF0000E046F120EF8
:10518000056F000E066F000E076F4EEC2CF001014C
:105190000A0E046F000E056F000E066F000E076FFB
:1051A0006EEC2CF0120E0C6E00C10BF00AEC0BF042
:1051B000130E0C6E01C10BF00AEC0BF0140E0C6E0A
:1051C00002C10BF00AEC0BF0150E0C6E03C10BF0D4
:1051D0000AEC0BF004017A0E826F73EC0EF00401FE
:1051E0002C0E826F73EC0EF00401370E826F73EC9D
:1051F0000EF004012C0E826F73EC0EF0D5EC26F04D
:10520000F2EF20F087C32AF188C32BF189C32CF178
:105210008AC32DF18BC32EF18CC32FF18DC330F1D6
:105220008EC331F190C332F191C333F10101296B87
:1052300086EC2DF0FDEC2CF0880E046F130E056F3C
:10524000000E066F000E076F42EC2CF0000E046F8C
:10525000040E056F000E066F000E076F4EEC2CF06B
:105260000101E80E046F800E056F000E066F000E40
:10527000076F6EEC2CF0060E0C6E00C10BF00AEC02
:105280000BF0070E0C6E01C10BF00AEC0BF0080ED0
:105290000C6E02C10BF00AEC0BF0090E0C6E03C190
:1052A0000BF00AEC0BF004017A0E826F73EC0EF037
:1052B00004012C0E826F73EC0EF00401380E826F25
:1052C00073EC0EF004012C0E826F73EC0EF067ECA1
:1052D00027F0F2EF20F007A8DEEF29F00101800EA1
:1052E000006F1A0E016F060E026F000E036F4BC1A6
:1052F00004F14CC105F14DC106F14EC107F13DEC81
:105300002CF003BF24EF2AF098EC2AF04BC100F1F7
:105310004CC101F14DC102F14EC103F107824AECCB
:105320002BF018C104F119C105F11AC106F11BC116
:1053300007F1F80E006FCD0E016F660E026F030EBF
:10534000036F3DEC2CF00E0E0C6E00C10BF00AEC5E
:105350000BF00F0E0C6E01C10BF00AEC0BF0100EEF
:105360000C6E02C10BF00AEC0BF0110E0C6E03C1B7
:105370000BF00AEC0BF00784010138EC2DF057C15B
:1053800000F158C101F107940A0E0C6E00C10BF038
:105390000AEC0BF00B0E0C6E01C10BF00AEC0BF0DB
:1053A0000C0E0C6E02C10BF00AEC0BF00D0E0C6E25
:1053B00003C10BF00AEC0BF024EF2AF007AA24EF4C
:1053C0002AF00784010138EC2DF057C100F158C1D3
:1053D00001F10794060E0C6E00C10BF00AEC0BF005
:1053E000070E0C6E01C10BF00AEC0BF0080E0C6EF0
:1053F00002C10BF00AEC0BF0090E0C6E03C10BF0AE
:105400000AEC0BF0078462C100F163C101F164C1D1
:1054100002F165C103F10794120E0C6E00C10BF08E
:105420000AEC0BF0130E0C6E01C10BF00AEC0BF042
:10543000140E0C6E02C10BF00AEC0BF0150E0C6E84
:1054400003C10BF00AEC0BF00798079A0401805196
:1054500081197F0B0DE09EA8FED714EE00F081515C
:105460007F0BE126E750812B0F01AD6E26EF2AF06E
:1054700005012F51010A13E081AA60EF2AF005010E
:105480002F51000A0AE00FB84FEF2AF005013067EC
:105490004FEF2AF00FB84FEF2AF0F8EF33F081B852
:1054A00060EF2AF068EC2EF060EF2AF0602F60EFDA
:1054B0002AF05FC560F50501010E306F3C0E316FBB
:1054C000BAEF0DF018C100F119C101F11AC102F1D2
:1054D0001BC103F1000E046F000E056F010E066F75
:1054E000000E076F6EEC2CF029A18DEF2AF02051F1
:1054F000D8B48DEF2AF018C100F119C101F11AC119
:1055000002F11BC103F1000E046F000E056F0A0EBD
:10551000066F000E076F6EEC2CF0120001010451B3
:105520000013055101130651021307510313120012
:105530000101186B196B1A6B1B6B12002AC182F4E4
:105540000401300E822773EC0EF02BC182F40401AB
:10555000300E822773EC0EF02CC182F40401300E61
:10556000822773EC0EF02DC182F40401300E8227E5
:1055700073EC0EF02EC182F40401300E822773EC1E
:105580000EF02FC182F40401300E822773EC0EF06E
:1055900030C182F40401300E822773EC0EF031C169
:1055A00082F40401300E822773EC0EF032C182F4D3
:1055B0000401300E822773EC0EF033C182F4040133
:1055C000300E822773EC0EF012002FC182F404011A
:1055D000300E822773EC0EF030C182F40401300EDD
:1055E000822773EC0EF031C182F40401300E822761
:1055F00073EC0EF032C182F40401300E822773EC9A
:105600000EF033C182F40401300E822773EC0EF0E9
:105610001200060E1E6E060E1F6E060E206E1E2E49
:105620000FEF2BF01F2E0FEF2BF0202E0FEF2BF094
:105630008B84020E1E6E020E1F6E020E206E1E2E38
:105640001FEF2BF01F2E1FEF2BF0202E1FEF2BF044
:105650008B941200FF0E1F6E1FC020F0030E1E6EF3
:105660008B841E2E30EF2BF0030E1E6E202E30EF9B
:105670002BF08B941FC020F0030E1E6E1E2E3EEFEB
:105680002BF0030E1E6E203E3EEF2BF01F2E2CEF54
:105690002BF012000101005305E1015303E1025315
:1056A00001E1002B0DEC2CF038EC2DF03951006F9E
:1056B0003A51016F420E046F4B0E056F000E066FDC
:1056C000000E076F4EEC2CF000C104F101C105F192
:1056D00002C106F103C107F118C100F119C101F1BE
:1056E0001AC102F11BC103F107B27BEF2BF042ECB0
:1056F0002CF07DEF2BF03DEC2CF000C118F101C136
:1057000019F102C11AF103C11BF1120038EC2DF09E
:1057100059C100F15AC101F1060E21EC0BF0E8CF9E
:1057200004F1070E21EC0BF0E8CF05F1080E21EC97
:105730000BF0E8CF06F1090E21EC0BF0E8CF07F1F2
:105740003DEC2CF000C124F101C125F102C126F18C
:1057500003C127F1290E046F000E056F000E066FBE
:10576000000E076F4EEC2CF0EE0E046F430E056F2B
:10577000000E066F000E076F42EC2CF024C104F1FE
:1057800025C105F126C106F127C107F14EEC2CF029
:1057900000C11CF101C11DF102C11EF103C11FF1C5
:1057A000120E21EC0BF0E8CF04F1130E21EC0BF0FC
:1057B000E8CF05F1140E21EC0BF0E8CF06F1150E41
:1057C00021EC0BF0E8CF07F10D0E006F000E016F1A
:1057D000000E026F000E036F4EEC2CF0180E046FDB
:1057E000000E056F000E066F000E076F6EEC2CF0BA
:1057F0001CC104F11DC105F11EC106F11FC107F155
:1058000042EC2CF06A0E046F2A0E056F000E066F34
:10581000000E076F3DEC2CF01200BF0EFA6E200E4A
:105820003A6F396BD8900037013702370337D8B059
:105830001EEF2CF03A2F13EF2CF039073A070353E1
:10584000D8B412000331070B80093F6F03390F0BE7
:10585000010F396F80EC5FF0406F390580EC5FF02D
:10586000405D405F396B3F33D8B0392739333FA9AA
:1058700033EF2CF040513927120001015DEC2DF07F
:10588000D8B01200010103510719346F20EC2DF03C
:10589000D8900751031934AF800F12000101346B07
:1058A00044EC2DF0D8A05AEC2DF0D8B012002FEC1B
:1058B0002DF038EC2DF01F0E366F70EC2DF00B35FF
:1058C000D8B020EC2DF0D8A00335D8B01200362F78
:1058D0005DEF2CF034B147EC2DF012000101346B78
:1058E00004510511061107110008D8A044EC2DF051
:1058F000D8A05AEC2DF0D8B01200086B096B0A6BD7
:105900000B6B70EC2DF01F0E366F70EC2DF0075105
:105910000B5DD8A498EF2CF006510A5DD8A498EF3F
:105920002CF00551095DD8A498EF2CF00451085DC6
:10593000D8A0ABEF2CF00451085F0551D8A0053D6D
:10594000095F0651D8A0063D0A5F0751D8A0073D60
:105950000B5FD8900081362F85EF2CF034B147ECE7
:105960002DF0346B44EC2DF0D89074EC2DF00751F1
:105970000B5DD8A4C8EF2CF006510A5DD8A4C8EF7F
:105980002CF00551095DD8A4C8EF2CF00451085D36
:10599000D8A0D7EF2CF0003FD7EF2CF0013FD7EF86
:1059A0002CF0023FD7EF2CF0032BD8B4120034B107
:1059B00047EC2DF012000101346B44EC2DF0D8B00F
:1059C000120079EC2DF0200E366F003701370237C8
:1059D000033711EE33F00A0E376FE7360A0EE75C35
:1059E000D8B0E76EE552372FEDEF2CF0362FE5EF0C
:1059F0002CF034B12981D890120001010A0E346FC5
:105A0000200E366F11EE29F03451376F0A0ED89000
:105A1000E652D8B0E726E732372F08EF2DF00333F0
:105A2000023301330033362F02EF2DF0E750FF0F22
:105A3000D8A00335D8B0120029B147EC2DF01200E0
:105A4000045100270551D8B0053D01270651D8B0B3
:105A5000063D02270751D8B0073D03271200005129
:105A6000086F0151096F02510A6F03510B6F120049
:105A70000101006B016B026B036B12000101046BEF
:105A8000056B066B076B12000335D8A0120003519B
:105A9000800B001F011F021F031F003F57EF2DF057
:105AA000013F57EF2DF0023F57EF2DF0032B342B22
:105AB000032512000735D8A012000751800B041FE0
:105AC000051F061F071F043F6DEF2DF0053F6DEF0B
:105AD0002DF0063F6DEF2DF0072B342B072512001C
:105AE0000037013702370337083709370A370B37D2
:105AF00012000101296B2A6B2B6B2C6B2D6B2E6B0B
:105B00002F6B306B316B326B336B120001012A51FA
:105B10000F0B2A6F2B510F0B2B6F2C510F0B2C6F70
:105B20002D510F0B2D6F2E510F0B2E6F2F510F0B71
:105B30002F6F30510F0B306F31510F0B316F3251CE
:105B40000F0B326F33510F0B336F120010A806D0BA
:105B50008994000EC76E220EC66E05D08984000E91
:105B6000C76E220EC66E050EE82EFED7120010A8D4
:105B700002D0898401D08994050EE82EFED7120048
:105B8000A6EC2DF09E96C69E000EC96EFF0E9EB628
:105B900002D0E82EFCD79E96C69E000EC96EFF0E60
:105BA0009EB602D0E82EFCD7C9CFAFF59E96C69E12
:105BB000000EC96EFF0E9EB602D0E82EFCD7C9CFEC
:105BC000B0F59E96C69E000EC96EFF0E9EB602D020
:105BD000E82EFCD7C9CFB1F59E96C69E000EC96EC1
:105BE000FF0E9EB602D0E82EFCD7C9CFB2F59E9626
:105BF000C69E000EC96EFF0E9EB602D0E82EFCD7E0
:105C0000C9CFB3F59E96C69E000EC96EFF0E9EB616
:105C100002D0E82EFCD7C9CFB4F59E96C69E000EE2
:105C2000C96EFF0E9EB602D0E82EFCD7C9CFB5F5DF
:105C3000B7EC2DF01200A6EC2DF09E96C69E800EBD
:105C4000C96EFF0E9EB602D0E82EFCD79E96C69E69
:105C5000AFC5C9FFFF0E9EB602D0E82EFCD79E96B8
:105C6000C69EB0C5C9FFFF0E9EB602D0E82EFCD777
:105C70009E96C69EB1C5C9FFFF0E9EB602D0E82E05
:105C8000FCD79E96C69EB2C5C9FFFF0E9EB602D037
:105C9000E82EFCD79E96C69EB3C5C9FFFF0E9EB6E2
:105CA00002D0E82EFCD79E96C69EB4C5C9FFFF0E53
:105CB0009EB602D0E82EFCD79E96C69EB5C5C9FFFB
:105CC000FF0E9EB602D0E82EFCD7B7EC2DF01200E6
:105CD000A6EC2DF09E96C69E070EC96EFF0E9EB6D0
:105CE00002D0E82EFCD79E96C69E000EC96EFF0E0F
:105CF0009EB602D0E82EFCD7C9CFAFF59E96C69EC1
:105D0000000EC96EFF0E9EB602D0E82EFCD7C9CF9A
:105D1000B0F59E96C69E000EC96EFF0E9EB602D0CE
:105D2000E82EFCD7C9CFB1F59E96C69E000EC96E6F
:105D3000FF0E9EB602D0E82EFCD7C9CFB2F5B7EC65
:105D40002DF0A6EC2DF09E96C69E22C0C9FFFF0E38
:105D50009EB602D0E82EFCD79E96C69E000EC96E57
:105D6000FF0E9EB602D0E82EFCD7C9CFB6F5B7EC31
:105D70002DF01200A6EC2DF09E96C69E870EC96EE1
:105D8000FF0E9EB602D0E82EFCD79E96C69EAFC5EB
:105D9000C9FFFF0E9EB602D0E82EFCD79E96C69E87
:105DA000B0C5C9FFFF0E9EB602D0E82EFCD79E9666
:105DB000C69EB1C5C9FFFF0E9EB602D0E82EFCD725
:105DC0009E96C69EB2C5C9FFFF0E9EB602D0E82EB3
:105DD000FCD7B7EC2DF0A6EC2DF09E96C69E23C006
:105DE000C9FFFF0E9EB602D0E82EFCD79E96C69E37
:105DF000B6C5C9FFFF0E9EB602D0E82EFCD7B7ECA1
:105E00002DF01200A6EC2DF09E96C69E870EC96E50
:105E1000FF0E9EB602D0E82EFCD79E96C69E000EC0
:105E2000C96EFF0E9EB602D0E82EFCD79E96C69E87
:105E3000800EC96EFF0E9EB602D0E82EFCD79E964D
:105E4000C69E800EC96EFF0E9EB602D0E82EFCD70D
:105E50009E96C69E800EC96EFF0E9EB602D0E82E9C
:105E6000FCD7B7EC2DF01200A6EC2DF09E96C69E46
:105E7000870EC96EFF0E9EB602D0E82EFCD79E9606
:105E8000C69E000EC96EFF0E9EB602D0E82EFCD74D
:105E90009E96C69E000EC96EFF0E9EB602D0E82EDC
:105EA000FCD79E96C69E800EC96EFF0E9EB602D08F
:105EB000E82EFCD79E96C69E800EC96EFF0E9EB63B
:105EC00002D0E82EFCD7B7EC2DF0120010A817D0A6
:105ED000A6EC2DF09E96C69E8F0EC96EFF0E9EB646
:105EE00002D0E82EFCD79E96C69E000EC96EFF0E0D
:105EF0009EB602D0E82EFCD7B7EC2DF0120068EC6D
:105F00002EF0120010A82DD0A6EC2DF09E96C69E65
:105F100023C0C9FFFF0E9EB602D0E82EFCD79E9686
:105F2000C69E450EC96EFF0E9EB602D0E82EFCD767
:105F3000B7EC2DF0A6EC2DF09E96C69E8F0EC96E86
:105F4000FF0E9EB602D0E82EFCD79E96C69E000E8F
:105F5000C96EFF0E9EB602D0E82EFCD7B7EC2DF02E
:105F60001200A6EC2DF09E96C69E23C0C9FFFF0E20
:105F70009EB602D0E82EFCD79E96C69E010EC96E34
:105F8000FF0E9EB602D0E82EFCD7B7EC2DF0A6ECA3
:105F90002DF09E96C69E910EC96EFF0E9EB602D043
:105FA000E82EFCD79E96C69EA50EC96EFF0E9EB625
:105FB00002D0E82EFCD7B7EC2DF01200A6EC2DF0A5
:105FC0009E96C69E23C0C9FFFF0E9EB602D0E82E45
:105FD000FCD79E96C69E810EC96EFF0E9EB602D05D
:105FE000E82EFCD7B7EC2DF01200A6EC2DF09E9613
:105FF000C69E23C0C9FFFF0E9EB602D0E82EFCD776
:106000009E96C69E010EC96EFF0E9EB602D0E82E69
:10601000FCD7B7EC2DF01200A6EC2DF09E96C69E94
:10602000910EC96EFF0E9EB602D0E82EFCD79E964A
:10603000C69EA50EC96EFF0E9EB602D0E82EFCD7F6
:10604000B7EC2DF01200A6EC2DF09E96C69E910E98
:10605000C96EFF0E9EB602D0E82EFCD79E96C69E55
:10606000000EC96EFF0E9EB602D0E82EFCD7B7EC2C
:106070002DF012000501256B266B276B286B899A82
:10608000400EC76E200EC66E9E96C69E030EC96E4B
:10609000FF0E9EB602D0E82EFCD79E96C69E27C560
:1060A000C9FFFF0E9EB602D0E82EFCD79E96C69E74
:1060B00026C5C9FFFF0E9EB602D0E82EFCD79E96DD
:1060C000C69E25C5C9FFFF0E9EB602D0E82EFCD79E
:1060D0009E96C69EC952FF0E9EB602D0E82EFCD7F1
:1060E000898A0F01C950FF0A01E1120005012E51F2
:1060F000130A05E005012E51170A0CE012000501F4
:10610000F00E256FFF0E266F0F0E276F000E286F03
:1061100093EF30F00501F00E256FFF0E266FFF0E96
:10612000276F000E286F899A400EC76E200EC66E2C
:106130009E96C69E030EC96EFF0E9EB602D0E82E36
:10614000FCD79E96C69E27C5C9FFFF0E9EB602D0FD
:10615000E82EFCD79E96C69E26C5C9FFFF0E9EB6AA
:1061600002D0E82EFCD79E96C69E25C5C9FFFF0E1D
:106170009EB602D0E82EFCD79E96C69EC952FF0E50
:106180009EB602D0E82EFCD7898A0F01C950FF0ABB
:106190001DE005012E51130A05E005012E51170AD5
:1061A0000BE012000501000E256F000E266F100E89
:1061B000276F000E286F12000501000E256F000EDC
:1061C000266F000E276F010E286F12000501256B48
:1061D000266B276B286B05012E51130A05E005017C
:1061E0002E51170A0CE012000501000E216F000E5F
:1061F000226F080E236F000E246F08EF31F00501A7
:10620000000E216F000E226F800E236F000E246F90
:1062100021C500F122C501F123C502F124C503F116
:1062200025C504F126C505F127C506F128C507F1E6
:106230008EEC2AF000C125F501C126F502C127F533
:1062400003C128F5899A400EC76E200EC66E9E9631
:10625000C69E030EC96EFF0E9EB602D0E82EFCD776
:106260009E96C69E27C5C9FFFF0E9EB602D0E82E99
:10627000FCD79E96C69E26C5C9FFFF0E9EB602D0CD
:10628000E82EFCD79E96C69E25C5C9FFFF0E9EB67A
:1062900002D0E82EFCD79E96C69EC952FF0E9EB62F
:1062A00002D0E82EFCD7898AC950FF0A08E104C150
:1062B00025F505C126F506C127F507C128F5D890B3
:1062C000050124332333223321332151F00B216F75
:1062D000216772EF31F0226772EF31F0236772EFBE
:1062E00031F0246708EF31F00501100E2527E86A28
:1062F0002623E86A2723E86A28231200E86A0501B2
:106300002E51130A06E005012E51170A0BE0020E6A
:10631000120005012851000A03E12751F00B07E0A4
:10632000010E120005012851000A01E0010E1200C1
:1063300029C500F12AC501F12BC502F12CC503F1D5
:1063400025C504F126C505F127C506F128C507F1C5
:106350003DEC2CF003BF12007EEC31F0D8A410EF1E
:1063600032F0899A400EC76E200EC66E9E96C69E6B
:10637000060EC96EFF0E9EB602D0E82EFCD7898AA3
:10638000899A9E96C69E020EC96EFF0E9EB602D0D8
:10639000E82EFCD79E96C69E27C5C9FFFF0E9EB667
:1063A00002D0E82EFCD79E96C69E26C5C9FFFF0EDA
:1063B0009EB602D0E82EFCD79E96C69E25C5C9FF84
:1063C000FF0E9EB602D0E82EFCD79E96C69E000E0B
:1063D000C96EFF0E9EB602D0E82EFCD7898A899A34
:1063E0009E96C69E050EC96EFF0E9EB602D0E82E82
:1063F000FCD79E96C69EC952FF0E9EB602D0E82ECE
:10640000FCD7C9B0F9EF31F0898A0501100E2527B4
:10641000E86A2623E86A2723E86A282398EF31F000
:106420001200899A400EC76E200EC66E9E96C69EBA
:10643000060EC96EFF0E9EB602D0E82EFCD7898AE2
:10644000899A9E96C69EC70EC96EFF0E9EB602D052
:10645000E82EFCD7898A0501256B266B276B286BF4
:106460001200899A400EC76E200EC66E9E96C69E7A
:10647000050EC96EFF0E9EB602D0E82EFCD79E9682
:10648000C69EC952FF0E9EB602D0E82EFCD7C9CFD9
:1064900037F5898A1200899A400EC76E200EC66EA3
:1064A0009E96C69EB90EC96EFF0E9EB602D0E82E0D
:1064B000FCD7898A1200899A400EC76E200EC66EDC
:1064C0009E96C69EAB0EC96EFF0E9EB602D0E82EFB
:1064D000FCD7898AFF0EE82EFED712007EEC31F041
:1064E000D8A41200899A400EC76E200EC66E9E96E2
:1064F000C69E030EC96EFF0E9EB602D0E82EFCD7D4
:106500009E96C69E27C5C9FFFF0E9EB602D0E82EF6
:10651000FCD79E96C69E26C5C9FFFF0E9EB602D02A
:10652000E82EFCD79E96C69E25C5C9FFFF0E9EB6D7
:1065300002D0E82EFCD79E96C69EC952FF0E9EB68C
:1065400002D0E82EFCD7898A0F01C950FF0AD8A4CF
:106550006BEF33F00501FE0E376F30A03799C0ECBA
:106560002DF0AFC538F5B0C539F5B1C53AF5B2C5AE
:106570003BF5B3C53CF5B4C53DF5B5C53EF507845F
:10658000B6C166F1B7C167F1B8C168F1B9C169F1C7
:106590004BC14FF14CC150F14DC151F14EC152F1BF
:1065A00057C159F158C15AF11CEC21F000C13FF517
:1065B00001C140F502C141F503C142F50501616722
:1065C000E9EF32F06267E9EF32F06367E9EF32F04A
:1065D0006467EDEF32F0FAEF32F061C504F162C5A5
:1065E00005F163C506F164C507F13DEC2CF003BF6E
:1065F0006BEF33F059C143F55AC144F5B9C545F5C0
:10660000BAC546F507940501110E326F899A400EFE
:10661000C76E200EC66E9E96C69E060EC96EFF0EF3
:106620009EB602D0E82EFCD7898A899A9E96C69E8D
:10663000020EC96EFF0E9EB602D0E82EFCD79E96C3
:10664000C69E27C5C9FFFF0E9EB602D0E82EFCD716
:106650009E96C69E26C5C9FFFF0E9EB602D0E82EA6
:10666000FCD79E96C69E25C5C9FFFF0E9EB602D0DA
:10667000E82EFCD725EE37F0322F02D04BEF33F067
:106680009E96C69EDECFC9FFFF0E9EB602D0E82EB4
:10669000FCD73CEF33F0898A899A9E96C69E050EF8
:1066A000C96EFF0E9EB602D0E82EFCD79E96C69EFF
:1066B000C952FF0E9EB602D0E82EFCD7C9B056EFE5
:1066C00033F0898A0501100E2527E86A2623E86A37
:1066D0002723E86A2823120021C500F122C501F111
:1066E00023C502F124C503F1899A400EC76E200E1E
:1066F000C66E9E96C69E0B0EC96EFF0E9EB602D04B
:10670000E82EFCD79E96C69E02C1C9FFFF0E9EB61C
:1067100002D0E82EFCD79E96C69E01C1C9FFFF0E8F
:106720009EB602D0E82EFCD79E96C69E00C1C9FF39
:10673000FF0E9EB602D0E82EFCD79E96C69EC9528A
:10674000FF0E9EB602D0E82EFCD725EE37F00501ED
:10675000100E326F9E96C69EC952FF0E9EB602D094
:10676000E82EFCD7C9CFDEFF322FAAEF33F0898A9B
:106770001200899A400EC76E200EC66E9E96C69E67
:10678000900EC96EFF0E9EB602D0E82EFCD79E96E4
:10679000C69E000EC96EFF0E9EB602D0E82EFCD734
:1067A0009E96C69E000EC96EFF0E9EB602D0E82EC3
:1067B000FCD79E96C69E000EC96EFF0E9EB602D0F6
:1067C000E82EFCD79E96C69EC952FF0E9EB602D0FA
:1067D000E82EFCD7C9CF2DF59E96C69EC952FF0E56
:1067E0009EB602D0E82EFCD7C9CF2EF5898A1200BA
:1067F00009EC2BF0B9C5E8FFD70802E309EC2BF050
:10680000B9C5E8FFC80802E309EC2BF0B9C5E8FFF9
:10681000B90802E309EC2BF0B9C5E8FFAA0802E3C6
:1068200009EC2BF0B9C5E8FF9B0802E309EC2BF05B
:106830004BEC32F0F29CF29E8B94C69AC2909482FA
:10684000948C720ED36ED3A4FED789968A909390BF
:10685000F29AF2949D909E909D929E92F298F2925E
:1068600066EC2FF0FF0EE8CF00F0E82EFED7002EEA
:10687000FCD7F290F286815081A841EF34F0F29E6D
:106880000300700ED36EF296F290010E306E03800C
:086890002AEC2BF056EF0BF08F
:10BF0000E844F926000C160C2B0C3F0C520C640C68
:10BF1000760C860C960CA50CB30CC10CCF0CDC0C6B
:06BF2000E80CF40C000C1B
:0200000400F00A
:0100C800FE39
:00000001FF
